:0400000002001E32AA
:03000B000238AB0D
:0100130032BA
:03001B00023E6A38
:0300FB000200FE02
:0300FE0002090DE7
:06010100C20D1260909097
:09010700746B75F0801260B512F2
:0E01100064DFAA82AB83ACF074E6C0E0740139
:0E011E00C0E08A828B838CF012171C158115AD
:06012C0081A20C9228C024
:0501320025121B1DD089
:0601370025E4A22833FAC2
:0C013D00E4A20C33FBEAB5032D7582052B
:0E014900C0021220DED002C002121B27D0021C
:0E015700C002121B4AD002C296D29690000A35
:0C016500C0021218BFD0023009CE758213
:0201710000226A
:06017300A20B9229E4A298
:030179002933FA2D
:0A017C00E4A20B33FBEAB5033DE5F6
:0C0186003230E60F90747475F080C002F7
:070192001216D2D002800D0D
:0D01990090747D75F080C0021216D2D00265
:0E01A600C296D296900032C0021218BFD0024C
:0701B40030090475820022EE
:0701BB00300DBE7582002229
:0601C200A20C9228E4A249
:0301C8002833FADF
:0C01CB00E4A20C33FBEAB5035AC0021298
:0D01D7006090D00290748675F080C0021216
:0A01E40060B5D002853C82C0021213
:0D01EE006251D00290748A75F080C0021238
:0E01FB0060B5D002C0021264DFAB82AC83ADEF
:0E020900F0D0028B828C838DF0C0021216D2D0
:0E021700D002C296D2969000C8C0021218BF44
:09022500D002300DA17582002207
:0A022E00C3E53C941550030201C221
:06023800200F030201C2C9
:06023E00A20C9228E4A2CC
:030244002833FA62
:0C024700E4A20C33FBEAB50361C0021214
:0A0253006090D002E53230E60F9013
:0E025D00748E75F080C0021260B5D002800D64
:0D026B0090749575F080C0021260B5D0024D
:0C027800853C82C002126251D002C0021C
:0E0284001264DFAB82AC83ADF0D0028B828CB3
:0E029200838DF0C0021216D2D002C296D29610
:0C02A000900032C0021218BFD002300DD6
:0502AC009A758200229A
:0A02B100C3E53C941D500302023E19
:0602BB00A20C9228E4A24F
:0302C1002833FAE5
:0B02C400E4A20C33FBEAB50302800348
:0302CF0002034ADD
:0C02D200C002126090D002E53230E60F4E
:0E02DE0090749C75F080C0021260B5D0028052
:0102EC000D04
:0D02ED009074A075F080C0021260B5D002C0
:0C02FA00853B82C002126251D002758266
:0C0306003AC00212609BD002853C82C00D
:0E03120002126251D002C0021264DFAB82AC54
:0E03200083ADF0D0028B828C838DF0C0021270
:0E032E0016D2D002C296D296900032C00212B1
:08033C0018BFD002200D0302DE
:0203440002C4F1
:04034600758200229A
:0A034A00C3E53C942450030202BBFB
:07035400126090853A82C09F
:04035B003CC03B1255
:0E035F0063E4158115811264DFAA82AB83ACC2
:0E036D00F01216D2C296D2969003201218BF3C
:0E037B00121B1D74B4C0E07401C0E09074A4A5
:0A03890075F08012171C1581158114
:0A039300C3E53C942A5048A20C92E6
:06039D0028E4A22833FA57
:0A03A300E4A20C33FBEAB503E7E522
:0C03AD003230E60F9074AD75F080C00295
:0703B9001216D2D002800DE4
:0D03C0009074B675F080C0021216D2D00203
:0E03CD00C296D296900032C0021218BFD00223
:0703DB00300DC57582002200
:0703E200126090853D8212BC
:0903E90062B39074BF75F080123C
:0C03F20060B51264DFAA82AB83ACF0128D
:0203FE0016D215
:0A040000C3E53C9432502AE5323087
:0D040A00E60B9074C675F0801216D28009C2
:090417009074CF75F0801216D22A
:0C042000C296D2969000321218BF300D28
:05042C00D375820022DF
:0A0431001260909074D875F08012EC
:06043B0060B5853E82124F
:0904410062519074DC75F0801228
:0C044A0060B51264DFAA82AB83ACF01234
:0804560016D29000FA1218BF43
:0A045E00C3E53C943A502AE5323021
:0D046800E60B9074E075F0801216D280094A
:090475009074E975F0801216D2B2
:0C047E00C296D2969000321218BF300DCA
:05048A00D37582002281
:0A048F001260909074F275F0801274
:0604990060B5853F8212F0
:0C049F0062511264DFAA82AB83ACF01241
:0904AB0016D29001F41218BFA250
:0504B4000C9228E4A2F7
:0304B9002833FAEB
:0C04BC00E4A20C33FBEAB50310C296D298
:0D04C80096900001C0021218BFD00280E71C
:0904D500A20C200E047582002225
:0904DE00C20E90003375F04012CB
:0E04E7002867121B1D74B4C0E07401C0E090C1
:0E04F50074F975F08012171C1581158174B40E
:0D050300C0E07401C0E090750275F0801238
:0A051000171C158115817582012268
:0A051A00C059858159058105811241
:0C0524001B1DAA590A7B007C40C002C0CD
:0E05300003C004758207122D5FAA8215811583
:0B053E00811581EA7005A859087605B8
:0C054900E5592402FA7B007C40C002C08F
:0E05550003C004758208122D5FAA821581155D
:0C056300811581EA7006A8590808761E70
:0D056F0075820A12195075820A12197DA8B2
:0C057C005908E624F6501C90750B75F031
:0E058800801216D27404C0E0E4C0E07582C098
:0905960012160C15811581801B61
:0E059F0090751475F0801216D27404C0E074CA
:0D05AD0001C0E07582C012160C1581158189
:0A05BA00E5592402FA7B007C40ADF5
:0C05C400590D7E007F40C002C003C0043F
:0E05D0008D828E838FF0122F03AA8215811563
:0905DE00811581EA70030209078E
:0A05E700758217121A51C2017A0042
:0A05F100A8590808B60015A859081B
:0C05FB0008763BA85908B600030207EA86
:06060700A8590816800549
:05060D00A859080816C1
:06061200A85908B6020021
:0B0618004010A8590808B60002800737
:07062300A8590808B61E0AE1
:0A062A00758201C0021219C2D0024D
:0D063400EA24FE501CC002126090D0028526
:070641003382C002C035C086
:0C064800341263E415811581D0021A8081
:010654005A4B
:0B065500C002126090D00230010F9034
:0E066000751D75F080C0021260B5D002800DCD
:0D066E0090752075F080C0021260B5D002BA
:0A067B00A85908A859088682C00299
:0E0685001262F5D00275823AC00212609BD05C
:0A06930002A8590808A859080886B3
:0E069D0082C002126282D002758220C0021258
:0406AB00609BD0027E
:0C06AF0030012AC0021264DFAB82AC8371
:0C06BB00ADF0D002C00274E6C0E0E4A282
:0B06C7000233C0E08B828C838DF012A8
:0A06D200171C15811581D002801A53
:0E06DC00C0021264DFAB82AC83ADF0D0028BA3
:0C06EA00828C838DF0C0021216D2D00268
:0606F600C201E531139280
:0606FC0000E4BA00010455
:01070200FBFB
:09070300EB604DA85908B60A008C
:0D070C005023C002C003E4C0E0758220123B
:0E071900155F1581D003D002758201C002C0A9
:0A07270003122057D003D0028022F5
:0E073100758200C002C003122057D003D00210
:0E073F00C002C0037401C0E075822012155F75
:06074D001581D003D0026B
:0E075300C002C003121B27D003D002C002C098
:0D07610003121B4AD003D002C296D296E5C7
:0A076E00396039E5592402FC8C02C1
:0C0778007B007E40AF590F7C007D40C02C
:0E07840002C003C0068F828C838DF0122F03FB
:0E079200AC82158115811581EC7003020907F8
:0A07A000758217121A517A008010BA
:0A07AA00E5315401FCE4A20033FD28
:0607B400B5040302070377
:0C07BA00C002121A5AE582D0026014A896
:0B07C6005908E624FF500C7582071252
:0707D1001A517A04D201D293
:0107D800021E
:0507D900BA01028003DB
:0307DE000205F120
:0707E100D201C2027A0002FE
:0207E80005F119
:0E07EA007401C0E075822112155F15817A003E
:0307F800BA040040
:0E07FB00501B75820FC00212197DD002C296EB
:0E080900D296900064C0021218BFD0020A807E
:01081700E000
:06081800C296D2967A039D
:0E081E00758214C002121950D002900014C04E
:0E082C00021218BFD002DAEAC296D296749673
:0D083A00C0E07401C0E090752375F08012DD
:08084700171C158115817A00D0
:03084F00BA0400E8
:0E085200501B75820FC00212197DD002C29693
:0E086000D296900064C0021218BFD0020A8027
:01086E00E0A9
:06086F00C296D2967A0346
:0E087500758214C002121950D002900014C0F7
:0E088300021218BFD002DAEAC296D29674961C
:0D089100C0E07401C0E090752C75F080127D
:08089E00171C158115817A0079
:0308A600BA040091
:0E08A900501B75820FC00212197DD002C2963C
:0E08B700D296900064C0021218BFD0020A80D0
:0108C500E052
:0608C600C296D2967A05ED
:0E08CC00758214C002121950D002900014C0A0
:0E08DA00021218BFD002DAEAC296D2967496C5
:0D08E800C0E07401C0E090750275F0801250
:0D08F500171C15811581758200121A7612EC
:050902002120121B1D65
:06090700855981D0592240
:0A090D00C0598581590581C296D2B8
:0B091700961238789000C81218BF122A
:0909220037711214F17582001204
:0C092B00145A75820112143B75820312ED
:0609370019C2122E141279
:0A093D002849E5827009121AC01261
:050947003771020AE215
:0C094C00AA590A7B007C40C002C003C016
:0E09580004758200122D5FAA8215811581158B
:0909660081EA6005A859088642E7
:0C096F00AA590A7B007C40C002C003C0F3
:0E097B0004758201122D5FAA82158115811567
:0B09890081EA6008A85908E624FF92EC
:010994001052
:0C099500AA590A7B007C40C002C003C0CD
:0E09A10004758202122D5FAA82158115811540
:0B09AF0081EA6008A85908E624FF92C6
:0109BA00112B
:0C09BB00AA590A7B007C40C002C003C0A7
:0E09C70004758203122D5FAA82158115811519
:0B09D50081EA6008A85908E624FF92A0
:0109E0001204
:0C09E100AA590A7B007C40C002C003C081
:0E09ED0004758205122D5FAA821581158115F1
:0B09FB0081EA6008A85908E624FF927A
:010A060013DC
:0C0A0700AA590A7B007C40C002C003C05A
:0E0A130004758206122D5FAA821581158115C9
:0B0A210081EA6008A85908E624FF9253
:010A2C0014B5
:0C0A2D00AA590A7B007C40C002C003C034
:0E0A390004758209122D5FAA821581158115A0
:090A470081EA6005A85908864304
:0C0A5000AA590A7B007C40C002C003C011
:0E0A5C000475820A122D5FAA8215811581157C
:090A6A0081EA6005A859088644E0
:0C0A7300AA590A7B007C40C002C003C0EE
:0E0A7F000475820B122D5FAA82158115811558
:090A8D0081EA6005A859088645BC
:0C0A9600AA590A7B007C40C002C003C0CB
:0E0AA20004758210122D5FAA82158115811530
:0B0AB00081EA6008A85908E624FF92C4
:010ABB001624
:0C0ABC00AA590A7B007C40C002C003C0A5
:0E0AC80004758211122D5FAA82158115811509
:0B0AD60081EA6008A85908E624FF929E
:010AE10017FD
:0E0AE2007406C0E07405C0E075820112160CA7
:0E0AF000158115817404C0E07406C0E07582A3
:0E0AFE000112160C158115817402C0E07407F8
:0D0B0C00C0E075820112160C158115819054
:0C0B1900012C1218BF90753575F0801289
:0E0B250016D2C296D2969007D01218BFC29672
:0E0B3300D2961214F19003E81218BFC296D2A7
:0E0B41009690753E75F0801216D29005DC126B
:0E0B4F0018BFC296D29674C8C0E07401C0E010
:0E0B5D0090754775F08012171C158115819058
:0E0B6B0005DC1218BFC296D2967496C0E074D4
:0E0B790001C0E090755075F08012171C1581B8
:0E0B870015817496C0E07401C0E09075597538
:0E0B9500F08012171C158115817496C0E07453
:0E0BA30001C0E090750275F08012171C1581DC
:0C0BB10015811214F19001F41218BF908D
:0C0BBD00003375F040122A05E582702D0F
:0B0BC900120101E58270142009119058
:0C0BD400756275F0801216D29004B01209
:040BE00018BF80E5D5
:0E0BE400758208121923758208121950758245
:040BF200081219C20A
:070BF600E543B4013F7A0062
:030BFD00BA030038
:0C0C0000E433FBA85908A602EB602FC2E9
:0E0C0C0096D296758200C002121A76D002901F
:0E0C1A000064C0021218BFD002758201C00231
:0E0C2800121A76D002900064C0021218BFD0DB
:040C3600020A80C36B
:0A0C3A00121B1D75820A121A51A840
:040C440059088602C3
:0E0C4800C0021226EBD002C002121A5AE58238
:0E0C5600D002602274035AFBBB0309C00212D5
:060C64002337D0028007D7
:070C6A00C0021225F1D002C7
:0B0C71000A758207C002121A51D0025F
:0A0C7C00E5426025E542B40155E5AC
:070C860039605475390020AC
:080C8D00084E20094BC00212C1
:0E0C9500051AD002758207C002121A51D00251
:020CA300803897
:080CA500E539603475390020C7
:080CAD00082E20092BC00212E1
:0E0CB5001B1DD002C00212548ED002C00212CB
:0E0CC3002120D002C002121B1DD00275820734
:090CD100C002121A51D002800386
:030CDA0075390069
:050CDD00100902805A1D
:0C0CE20020084DC002125BE4D002C002EA
:0B0CEE00126090D002853382C002C06B
:040CF90035C03412BC
:0E0CFD0063E415811581D002C0021264DFABE2
:0E0D0B0082AC83ADF0D002C00274DCC0E07494
:0E0D190001C0E08B828C838DF012171C1581B7
:0B0D27001581D002C002121B1DD0027B
:0A0D3200758207C002121A51D002A8
:0E0D3C00C002121B27D002C002121B4AD002B6
:0E0D4A00C002121C9AD002C00212227FD002F8
:0B0D5800C296D296020C48855981D04B
:020D6300592213
:09746B0046756E6B2020203F00E5
:097474002D2D203F3F202D2D009D
:09747D002D2D201212202D2D00EE
:047486002D2D200088
:04748A00202D2D0084
:07748E003F3F3A20203A00C5
:077495003F3F3A12123A00DA
:04749C0020203A0072
:0474A00012123A008A
:0974A4003F3F0B3F3F0B3F3F004F
:0974AD0020200B3F3F0B3F3F0084
:0974B60012120B3F3F0B3F3F0097
:0774BF000B3F3F0B3F3F00B4
:0974C60009090912120B3F3F00F5
:0974CF0009090920200B3F3F00D0
:0474D8000909090095
:0474DC000B3F3F0023
:0974E00009090909090912120049
:0974E90009090909090920200024
:0774F200090909090909005D
:0974F9002020204F6B162020001A
:0975020020202020202020200080
:09750B0020202D2D3A2D2D200029
:097514002020202D3A2D2D20002D
:03751D002020002B
:0375200009090056
:0975230020205A65697420200043
:09752C002020456E64652020005A
:0975350047656E756852200900DB
:09753E0056312E342030333200A6
:09754700A927303620766F6E0092
:097550005265696D617220200092
:0975590047726173626F6E20003D
:09756200D7D7D7D7D7D7D7D70068
:03007700752E07DC
:070D6500AA828A03BBA9006A
:050D6C005003020DDF41
:050D7100BA6002803FA2
:050D7600BAA902803261
:050D7B00BAB002803156
:050D8000BAB702803447
:050D8500BAC402803336
:050D8A00BAD602803220
:050D8F00BAD70280311B
:050D9400BADC02803012
:050D9900BADF02802F0B
:050D9E00BAE402802E02
:050DA300BAF602802DEC
:050DA800BAFC32802CB2
:040DAD007A08802E12
:040DB1007A9A802A80
:040DB5007A9B80267F
:040DB9007A9C80227E
:040DBD007A9D801E7D
:040DC1007A9E801A7C
:040DC5007A9F80167B
:040DC9007AA080127A
:040DCD007AA1800E79
:040DD1007AA2800A78
:040DD5007AA3800677
:040DD9007AA4800276
:020DDD007A009A
:0A0DDF00EA75F007A4246BFA74759E
:070DE90035F08A82F5832238
:0A0DF000C05985815905810581AACB
:0C0DFA0082A859181818E624F8500302CB
:020E06001435A1
:0A0E0800A959191919E72426F886E4
:0D0E120082C002120D65AB82AC83D002E5F8
:0C0E1F005924FCF88682C002C003C00405
:0E0E2B00120D65AD82AE83D004D003D002A8B4
:0A0E39005908A60508A606A85918D6
:0E0E43001818900000E6F0C374808AF063F087
:080E51008095F0400302111D21
:0E0E5900C3748A8AF063F08095F050027A0A22
:0E0E6700C3EA648094875014EA2BF582E43CC1
:0C0E7500F583E493FFE55924FCF8A60780
:020E8100803DB2
:0C0E8300C3EA6480948A5009E55924FCFD
:050E8F00F87600802C44
:0E0E9400C003C004EAFF3395E0FBEF24F6FF35
:0C0EA200EB34FFFBA85908EF26F582EBAB
:0C0EAE000836F583E493FBE55924FCF8BA
:060EBA00A603D004D003E2
:0C0EC000E55924FCF8902000E6F00AC37D
:0E0ECC00EA648094875014EA2BF582E43CF52A
:0C0EDA0083E493FFE55924FCF8A6078090
:010EE6003DCE
:0C0EE700C3EA6480948A5009E55924FC99
:050EF300F87600802CE0
:0E0EF800C003C004EAFF3395E0FBEF24F6FFD1
:0C0F0600EB34FFFBA85908EF26F582EB46
:0C0F12000836F583E493FBE55924FCF855
:060F1E00A603D004D0037D
:0C0F2400E55924FCF8902400E6F00AC314
:0E0F3000EA648094875014EA2BF582E43CF5C5
:0C0F3E0083E493FFE55924FCF8A607802B
:010F4A003D69
:0C0F4B00C3EA6480948A5009E55924FC34
:050F5700F87600802C7B
:0E0F5C00C003C004EAFF3395E0FBEF24F6FF6C
:0C0F6A00EB34FFFBA85908EF26F582EBE2
:0C0F76000836F583E493FBE55924FCF8F1
:060F8200A603D004D00319
:0C0F8800E55924FCF8902800E6F00AC3AC
:0E0F9400EA648094875014EA2BF582E43CF561
:0C0FA20083E493FFE55924FCF8A60780C7
:010FAE003D05
:0C0FAF00C3EA6480948A5009E55924FCD0
:050FBB00F87600802C17
:0E0FC000C003C004EAFF3395E0FBEF24F6FF08
:0C0FCE00EB34FFFBA85908EF26F582EB7E
:0C0FDA000836F583E493FBE55924FCF88D
:060FE600A603D004D003B5
:0C0FEC00E55924FCF8902C00E6F00AC344
:0E0FF800EA648094875014EA2BF582E43CF5FD
:0C10060083E493FFE55924FCF8A6078062
:011012003DA0
:0C101300C3EA6480948A5009E55924FC6B
:05101F00F87600802CB2
:0E102400C003C004EAFF3395E0FBEF24F6FFA3
:0C103200EB34FFFBA85908EF26F582EB19
:0C103E000836F583E493FBE55924FCF828
:06104A00A603D004D00350
:0C105000E55924FCF8903000E6F00AC3DB
:0E105C00EA648094875014EA2BF582E43CF598
:0C106A0083E493FFE55924FCF8A60780FE
:011076003D3C
:0C107700C3EA6480948A5009E55924FC07
:05108300F87600802C4E
:0E108800C003C004EAFF3395E0FBEF24F6FF3F
:0C109600EB34FFFBA85908EF26F582EBB5
:0C10A2000836F583E493FBE55924FCF8C4
:0610AE00A603D004D003EC
:0C10B400E55924FCF8903400E6F00AC373
:0E10C000EA648094875014EA2BF582E43CF534
:0C10CE0083E493FFE55924FCF8A607809A
:0110DA0035E0
:0C10DB00C3EA6480948A5009E55924FCA3
:0510E700F876008024F2
:0E10EC00EAFF3395E0FDEF24F6FFED34FFFD43
:0C10FA00A85908EF26F582ED0836F583B2
:0A110600E493FDE55924FCF8A6056A
:0B111000E55924FCF8903800E6F002DE
:02111B00143589
:0A111D00C3EA6480947650027AF66B
:0E112700C374798AF063F08095F05021EAFDE0
:0E1135003395E0FE74062DFDE43EFEED2BF535
:0C11430082EE3CF583E493FDE55924FCAA
:05114F00F8A605803840
:0D115400C374768AF063F08095F05009E5D1
:081161005924FCF876008023FC
:0E116900EAFD3395E0FE74102DFDE43EFEA875
:0C1177005908ED26F582EE0836F583E4F9
:0911830093FDE55924FCF8A605D2
:0C118C00E55924FCF8903800E6F01AC386
:0E11980074798AF063F08095F05021EAFD33FF
:0E11A60095E0FE74062DFDE43EFEED2BF58275
:0C11B400EE3CF583E493FDE55924FCF8C3
:0411C000A6058038C8
:0D11C400C374768AF063F08095F05009E561
:0811D1005924FCF8760080238C
:0E11D900EAFD3395E0FE74102DFDE43EFEA805
:0C11E7005908ED26F582EE0836F583E489
:0911F30093FDE55924FCF8A60562
:0C11FC00E55924FCF8903400E6F01AC31A
:0E12080074798AF063F08095F05021EAFD338E
:0E12160095E0FE74062DFDE43EFEED2BF58204
:0C122400EE3CF583E493FDE55924FCF852
:04123000A605803857
:0D123400C374768AF063F08095F05009E5F0
:081241005924FCF8760080231B
:0E124900EAFD3395E0FE74102DFDE43EFEA894
:0C1257005908ED26F582EE0836F583E418
:0912630093FDE55924FCF8A605F1
:0C126C00E55924FCF8903000E6F01AC3AD
:0E12780074798AF063F08095F05021EAFD331E
:0E12860095E0FE74062DFDE43EFEED2BF58294
:0C129400EE3CF583E493FDE55924FCF8E2
:0412A000A6058038E7
:0D12A400C374768AF063F08095F05009E580
:0812B1005924FCF876008023AB
:0E12B900EAFD3395E0FE74102DFDE43EFEA824
:0C12C7005908ED26F582EE0836F583E4A8
:0912D30093FDE55924FCF8A60581
:0C12DC00E55924FCF8902C00E6F01AC341
:0E12E80074798AF063F08095F05021EAFD33AE
:0E12F60095E0FE74062DFDE43EFEED2BF58224
:0C130400EE3CF583E493FDE55924FCF871
:04131000A605803876
:0D131400C374768AF063F08095F05009E50F
:081321005924FCF8760080233A
:0E132900EAFD3395E0FE74102DFDE43EFEA8B3
:0C1337005908ED26F582EE0836F583E437
:0913430093FDE55924FCF8A60510
:0C134C00E55924FCF8902800E6F01AC3D4
:0E13580074798AF063F08095F05021EAFD333D
:0E13660095E0FE74062DFDE43EFEED2BF582B3
:0C137400EE3CF583E493FDE55924FCF801
:04138000A605803806
:0D138400C374768AF063F08095F05009E59F
:081391005924FCF876008023CA
:0E139900EAFD3395E0FE74102DFDE43EFEA843
:0C13A7005908ED26F582EE0836F583E4C7
:0913B30093FDE55924FCF8A605A0
:0C13BC00E55924FCF8902400E6F01AC368
:0E13C80074798AF063F08095F05021EAFD33CD
:0E13D60095E0FE74062DFDE43EFEED2BF58243
:0C13E400EE3CF583E493FBE55924FCF893
:0413F000A603803799
:0D13F400C374768AF063F08095F05009E52F
:081401005924FCF8760080225A
:0D140900EA3395E0FB74102AFAE43BFBA8DF
:0C1416005908EA26F582EB0836F583E45D
:0914220093FAE55924FCF8A60236
:0A142B00E55924FCF8902000E6F0DB
:06143500855981D0592207
:0C143B00E582FA60107407552E90400006
:09144700D39407F4F0432E802237
:0A1450009040007407F0532E7F2235
:0E145A00E582FA24FC4056EA2A2A90146873B0
:0714680002147402147E025D
:05146F0014880214A125
:0A1474007480552E4407F52E8039D0
:0A147E007480552E4401F52E802FD6
:091488007407552EFABA0701227F
:0A1491007407552E2401FA748055EB
:06149B002E4AF52E80161A
:0914A1007407552EFABA0101226C
:0A14AA007407552E14FA7480552EB5
:0314B4004AF52EC8
:0A14B700E52E30E70C7407552E9067
:0714C1004000D39407F4F092
:0614C80030B30320B41B49
:0814CE00747F552EFABA0300E9
:0614D6005004D2B3C2B4C1
:0C14DC00747F552EFA24FB5004C2B3D2DA
:0114E800B44F
:0114E90022E0
:0714EA00747F552EF58222EC
:0214F1007A007F
:0314F300BA080034
:0D14F6005026900000EAF0902000E4F090F5
:0E1503002400F0902800F0902C00F0903000B2
:0D151100E4F0903400F0903800F00A80D52E
:0D151E009060007480F09064007481F09083
:0E152B0068007482F0906C007483F090700081
:0E1539007484F09074007485F09078007486CD
:09154700F0907C007487F07A003A
:03155000BA0800D6
:0B1553005009EA2426F876200A80F2F6
:01155E00226A
:08155F00C059858159AA82A838
:0C15670059181818E624F8500302160664
:0E1573008A82C002120D65AB82AC83D002A842
:0C15810059181818900000E6F08B828CBE
:0E158D0083E493FDA3AB82AC83902000EDF0CD
:0D159B008B828C83E493FDA3AB82AC839024
:0E15A8002400EDF08B828C83E493FDA3AB82D4
:0E15B600AC83902800EDF08B828C83E493FDD3
:0E15C400A3AB82AC83902C00EDF08B828C8365
:0E15D200E493FDA3AB82AC83903000EDF08B70
:0E15E000828C83E493FDA3AB82AC8390340035
:0E15EE00EDF08B828C83E493FB903800F0A824
:0A15FC0059181818E62426F8A60274
:06160600855981D0592234
:08160C00C059858159AA82E54D
:071614005924FCF8B60100A7
:09161B005007E55924FCF87601A2
:0B162400E55924FCF8E624F55007E52A
:06162F005924FCF8760AC4
:021635007B0038
:03163700BB3A00BB
:05163A0040030216B997
:0E163F00EB9079EE93FC20E721EC24F6FDC041
:0C164D0002C003C002A859181818E6C01B
:0E165900E08D82120DF015811581D003D002B4
:021667008028D9
:0A166900A859181818E62426F8A660
:0C16730002C002C0037420C0E0A8591897
:0E167F001818E6C0E08C82120DF0158115815E
:04168D00D003D002B4
:0C169100E55924FCF886047D00740BC3AE
:0E169D009CF582E49DF583C002C0031218BFC5
:0A16AB00D003D00220080720090434
:0416B5000B021637D7
:0B16B900A859181818E6C0E08A821239
:0C16C400155F1581C296D296855981D021
:0216D00059229D
:0E16D200AA82AB83ACF0BA0007BB0004BC00D8
:0216E0000122E5
:0216E2007D0089
:0316E400BD08003E
:0E16E70050328A828B838CF01273C9FE60260B
:0516F500BE090280198E
:0D16FA00C002C003C004C005C0058E8212EE
:0C170700155F1581D005D004D003D0027E
:051713000ABA00010B01
:031718000D80C978
:01171B0022AB
:0A171C00C059858159C082C083C006
:0C172600F0A85908B6000B08B600070830
:06173200B600030218B925
:021738007D0131
:0B173A00C3ED6480948A40030217E0B6
:06174500C3E49DFE7F00DD
:03174B00BF0800D4
:0C174E005068C006A85908EF26FEE40809
:0E175A0036FA0886038E828A838BF01273C9DA
:08176800FE8E04E4BC00010444
:09177000D0067044BC0902803C63
:0C177900A859181818E6601BC005C0062F
:0E178500C007C004C0078D82120DF01581153B
:0917930081D007D006D0058019B1
:0D179C00C005C006C007C004C0078E821241
:0C17A9000DF015811581D007D006D00589
:0317B5000F80930F
:0C17B800E55924FCF886027B0074FFC396
:0E17C4009AF582E49BF583C0051218BFD0058C
:0A17D200C296D296200807200904F1
:0417DC000D02173AA9
:0217E0007A008D
:0317E200BA080042
:0517E50040030218A3FF
:0C17EA00A85908EA26FBE40836FC088633
:0E17F600058B828C838DF01273C9FB8B04BCB3
:0518040000030218A31F
:0C180900BC090AEA2426F886038B048040
:0118150006CC
:06181600EA2426F8A604F6
:0E181C008C82C002120D65AB82AC83D00290AC
:0E182A000000EAF08B828C83E493FDA3AB8276
:0E183800AC83902000EDF08B828C83E493FD56
:0E184600A3AB82AC83902400EDF08B828C83E8
:0E185400E493FDA3AB82AC83902800EDF08BF3
:0E186200828C83E493FDA3AB82AC83902C00B8
:0E187000EDF08B828C83E493FDA3AB82AC83FE
:0E187E00903000EDF08B828C83E493FDA3ABE1
:0E188C0082AC83903400EDF08B828C83E49369
:09189A00FB903800F00A0217E28D
:0C18A300E55924FCF886027B0074FFC3AA
:0A18AF009AF582E49BF5831218BF3E
:0618B900855981D059227F
:0E756B000A150A150A150A0E0E041F040A114D
:0E757900181C1E1F1E1C1803070F1F0F0703F0
:0E75870010181C1E1C18100010181C181000E4
:0E7595000000101810000000000010000000A0
:0E75A3000E1F1117111F0E0000000000000047
:0E75B10000181800181800000000000000105C
:0E75BF00000E1111110E00000E1F1F1F0E00F6
:0E75CD00040E1F04040404040404041F0E042E
:0E75DB000004081F0804000004021F02040040
:0E75E9001F1F1F1F1F1F1F00000004000000B7
:0E75F7000000040E04000000040E1F0E04002D
:0E760500000000000000151F1F1F1F1F1F1F89
:0E7613001F11111111111F1F1F1F1F1F1F1FFD
:0E7621001F11171317171F1F1B131B1B111F01
:0E762F001F111D1117111F1F111D191D111FF5
:0E763D0000000000000000000000000000003F
:0E764B0000000000000000040404040004001D
:0E7659000A0A0000000000000A1F0A1F0A00B3
:0E766700040F140E051E041819020408130364
:0E7675000814140815120D0606040200000089
:0E7683000204080808040208040202020408B7
:0E769100000A041F040A000004041F04040081
:0E769F000000000C0C04080000001F0000009A
:0E76AD00000000000C0C000001020408100098
:0E76BB000E11111111110E040C040404040E22
:0E76C9000E11010608111F0E11010601110E0F
:0E76D700101012121F02021F101E0101110ED0
:0E76E5000E10101E11110E1F010102040404EC
:0E76F3000E11110E11110E0E11110F01020CCD
:0E770100000C0C000C0C000C0C000C0C04080E
:0E770F000102040804020100001F001F000018
:0E771D00100804020408100E110102040004FA
:0E772B000E11171517100E0E11111F1111114E
:0E7739001E11111E11111E0E11101010110E36
:0E7747001E11111111111E1F10101E10101F07
:0E7755001F10101C1010100E11101711110E25
:0E7763001111111F1111110E04040404040E63
:0E7771000101010101110E1112141814121160
:0E777F001010101010101F111B1515111111F4
:0E778D00111119151311110E11111111110EF8
:0E779B001E11111E1010100E11111115120DDD
:0E77A9001E11111E1412110E11100E01110EE0
:0E77B7001F0404040404041111111111110E19
:0E77C5001111110A0A040411111115151B11DE
:0E77D30011110A040A111111110A0404040410
:0E77E1001F01020408101F0E08080808080EF9
:0E77EF00001008040201000E02020202020E47
:0E77FD00040A11000000000000000000001F40
:0E780B000606040200000000000E010F110F1F
:0E7819001010161911191600000E1110110E84
:0E78270001010D1311130D00000E111F100EA4
:0E7835000609081E08080800000F110F010EBA
:0E784300101016191111110400000C04040E8F
:0E7851000200060202120C0808090A0C0A09BD
:0E785F000C04040404040E00001A151515157F
:0E786D000000161911111100000E1111110E5C
:0E787B0000001E1119161000000E11130D0151
:0E78890000000B0C08080800000E100E011E77
:0E78970004040F040404030000111111130D6A
:0E78A50000001111110A040000111115150A3E
:0E78B3000000110A040A11000011110F010E4D
:0E78C10000001F0204081F0204040804040251
:0E78CF0004040404040404080404020404086D
:0E78DD0008150200000000000000010000007D
:0E78EB00000002020200000002040504020078
:0E78F90004080A0A0A080408121415141208DA
:0E79070000000010000000000008080800004A
:0E7915000008041404080004020A0A0A02040E
:0E792300020905150509021F11111111111F8E
:0E793100040404040404041F01011F10101FAD
:0E793F001F01010F01011F1212121F0202028E
:0E794D001F10101F01011F1F10101F11111F0E
:0E795B001F0101010101011F11111F11111F58
:0E7969001F11111F010101000E000000000E91
:0E7977000006010000100C00020101101008B3
:0E79850000000111111000000010111101008E
:0E79930000081010010102000C100000010697
:0E79A100060909060000000C0C040800000096
:0E79AF00000000040000000A000E111F11115C
:0E79BD000A000E1111110E00110A040A110029
:0E79CB000A00111111110E0C121611111610D6
:0E79D9000A000E010F110F0A000E1111110EFF
:0779E7000A00111111130D3C
:0E79EE0009070604030100FFFDFCFBFBFAFA8B
:0E79FC00FAFAFAFBFBFCFDFEFEFF00010102A1
:0E7A0A0002030303030303030302020101004E
:0E7A180000FFFFFFFEFEFEFEFEFEFEFFFFFF74
:027A2600FF005F
:07007A00754C00754D807507
:060081004E007531FA7516
:0600870033007534007522
:06008D0035007536017517
:060093003701753800750D
:06009900390075403575C9
:06009F00410475420075EA
:0600A500430075440875DC
:0600AB004500754601C28C
:0400B10003C204C2C0
:0400B50005C206C2B8
:0400B90007C208C2B0
:0400BD0009C20AC2A8
:0400C1000DC20EC29C
:0400C5000FD210D274
:0400C90011D212D26C
:0400CD0013D214C274
:0400D10015D216D25C
:0100D5001713
:0418BF00AA82AB83CB
:0718C300BA0004BB00012282
:0E18CA00C3EA94F4EB94015023D310AF01C392
:0A18D800C0D08A2F8B30D0D092AF21
:0418E2007A007B000D
:0818E600AC30BC00FBAC2FE5A7
:0818EE00307D00BC00F280CD4A
:0518F600D310AF01C397
:0A18FB00C0D0752FF4753001D0D075
:0A19050092AFEA240CFAEB34FEFB6B
:08190F00AC30BC00FBAC2FE57D
:0C191700307D00BC00F2C296D29680A089
:0A192300E582FA75F00AA4FAC2AFDB
:05192D00BA0002801B5E
:021932007B0038
:03193400BB1500E0
:071937005005D2920B80F66F
:02193E007B002C
:03194000BB1500D4
:071943005005C2920B80F673
:03194A001A80E020
:03194D00D2AF22F4
:0A195000E582FA75F00AA4FAC2AFAE
:05195A00BA0002801B31
:02195F007B000B
:03196100BB1100B7
:071964005005D2920B80F642
:02196B007B00FF
:03196D00BB1100AB
:071970005005C2920B80F646
:031977001A80E0F3
:03197A00D2AF22C7
:0A197D00E582FA75F00AA4FAC2AF81
:05198700BA00028033EC
:02198C007B00DE
:03198E00BB090092
:071991005005D2920B80F615
:021998007B00D2
:03199A00BB090086
:07199D005005C2920B80F619
:0219A4007B00C6
:0319A600BB09007A
:0719A9005005D2920B80F6FD
:0219B0007B00BA
:0319B200BB09006E
:0719B5005005C2920B80F601
:0319BC001A80C8C6
:0319BF00D2AF2282
:0A19C200E582FA75F00AA4FAC2AF3C
:0619CC00BA0003021A4EEE
:0219D2007B0098
:0319D400BB06004F
:0719D7005005D2920B80F6CF
:0219DE007B008C
:0319E000BB060043
:0719E3005005C2920B80F6D3
:0219EA007B0080
:0319EC00BB060037
:0719EF005005D2920B80F6B7
:0219F6007B0074
:0319F800BB06002B
:0719FB005005C2920B80F6BB
:021A02007B0067
:031A0400BB06001E
:071A07005005D2920B80F69E
:021A0E007B005B
:031A1000BB060012
:071A13005005C2920B80F6A2
:021A1A007B004F
:031A1C00BB060006
:071A1F005005D2920B80F686
:021A26007B0043
:031A2800BB0600FA
:071A2B005005C2920B80F68A
:021A32007B0037
:031A3400BB0600EE
:071A37005005D2920B80F66E
:021A3E007B002B
:031A4000BB0600E2
:071A43005005C2920B80F672
:041A4A001A0219CC97
:031A4E00D2AF22F2
:051A510085824785318C
:041A560048C2182248
:071A5A00201812E531C395CD
:091A610048FAC3E5479A5004D28B
:031A6A00188002DF
:021A6D00C2189D
:071A6F00E4A21833F5822206
:071A7600AA82BA00028005FC
:051A7D00BA011F800703
:071A8200C215D2B3D2B42259
:0A1A8900C2151214EAAA82BA040082
:071A93005005D2B3C2B422DA
:051A9A00C2B3D2B4222A
:031A9F00D215223B
:061AA200E582FAB4010028
:031AA80092B722D0
:061AAB00E582FAB401001F
:071AB10092B58A82021AA21D
:081AB800A2B5B3E433F582226C
:0B1AC000907A2875F0801216D27A0090
:031ACB00BAC80096
:0E1ACE00504CEA30E512C0027406C0E075828A
:0A1ADC003F12155F1581D002801043
:0E1AE600C0027406C0E075822012155F1581E3
:021AF400D0021E
:0E1AF60090000AC0021218BFD002C296D2960B
:0E1B0400C002123771D002C002122849D0026E
:0A1B1200C002122E14D0020A80AFA8
:011B1C0022A6
:061B1D00C205753900C28B
:041B230008C20922C9
:0A1B2700E532235401FAE4A2193359
:051B3100FBB5020122DA
:0A1B3600E5323392193097067582EC
:041B40000202145A2F
:061B440075820302145A31
:061B4A00E543B402012294
:071B5000200804200501221A
:051B5700C208C20520D8
:031B5C0012012251
:0E1B5F001214F175820C12197DC296D29620D6
:051B6D00B503021BF4AA
:0E1B7200758201121AAB7402C0E07582451232
:0E1B8000155F15817403C0E075826912155F50
:0E1B8E0015817404C0E075826E12155F15811A
:0E1B9C007406C0E075820C12155F15817A0088
:031BAA00BA04007A
:051BAD004003021C735F
:0E1BB200758200C002121AA2D002900078C004
:0E1BC000021218BFD002BA0210C0027406C092
:0B1BCE00E075820D12155F1581D0023A
:0E1BD900758201C002121AA2D002900078C0DC
:0D1BE700021218BFD002C296D2960A80B634
:0E1BF400758200121AAB7402C0E075824112B5
:0E1C0200155F15817403C0E075827512155FC1
:0E1C100015817404C0E075827312155F158192
:0E1C1E007406C0E075820D12155F15817A0004
:031C2C00BA0400F7
:0D1C2F005042758201C002121AA2D002902C
:0E1C3C000078C0021218BFD002BA0210C00217
:0E1C4A007406C0E075820C12155F1581D00281
:0E1C5800758200C002121AA2D002900078C05D
:0D1C6600021218BFD002C296D2960A80B9B1
:0E1C7300121B1D1264DFAA82AB83ACF074F06A
:0D1C8100C0E07401C0E08A828B838CF012F9
:0C1C8E00171C15811581758207021A5180
:0A1C9A00C0598581590581058105B7
:081CA40081E543B40102801345
:081CAC00E543B40203021E8DA2
:081CB400E543B40403021F7AAA
:031CBC0002201DE6
:071CBF00E533B54402800388
:031CC600022020D9
:071CC900E534B5450280037C
:031CD000022020CF
:0A1CD300C3E535940A400302202007
:0A1CDD00754618AA590A7B007C40E6
:0D1CE700C002C003C00490003675F040122A
:081CF40072E2158115811581D2
:0C1CFC00AA590A7B007C408A828B838CF2
:0C1D0800F012692EAA590A7B007C408A68
:0C1D1400828B838CF0126B65AA82C228BF
:081D20002017178A82C025126A
:0B1D280070EBE582D025600A741825DE
:041D330046F546D259
:031D370028803FC2
:0A1D3A0020163CAA590A7B007C40E9
:0C1D44008A828B838CF0C0251265A9AA4E
:081D500082D025BA06028019B9
:0C1D5800AA590A7B007C408A828B838C95
:091D6400F0C0251265A9AA82D085
:041D6D0025BA070884
:071D710074182546F546D267
:011D78002842
:061D7900302803021CFCEF
:071D7F00E54624F3F54630B0
:051D86001303021E1E04
:0A1D8B00121AB8E5827003021E1E52
:0E1D95007582031219C27496C0E07401C0E09A
:0E1DA300907A3175F08012171C158115819011
:0E1DB10003201218BF74B4C0E07401C0E090AB
:0E1DBF007A3A75F08012171C1581158174B4E4
:0D1DCD00C0E07401C0E0907A4375F0801210
:0E1DDA00171C1581158174B4C0E07401C0E0BF
:0E1DE800907A4C75F08012171C1581158190B1
:0E1DF60001F41218BF758200121A7674F0C044
:0E1E0400E07401C0E0907A5575F08012171C52
:0A1E120015811581754B007543041E
:021E1C008066DE
:0A1E1E00744BC0E07400C0E0744093
:0E1E2800C0E0758204122D5FAA82158115811B
:0B1E36001581EA7006754B14121AC0EB
:0C1E41007582FF121A76D20A75821912FF
:0E1E4D00195075821912197D7496C0E0740147
:0E1E5B00C0E0907A5E75F08012171C1581159C
:0C1E6900813013087582191219238006BD
:061E7500758201121AAB98
:091E7B009003E81218BF75430240
:091E8400758207121A5102202098
:0A1E8D00301341E532235401FAE45A
:091E9700A21A33FBB502028031EE
:0A1EA000E53233921AC296D296750D
:0E1EAA00820A12197D9000641218BF7582071B
:0E1EB8001219C2C296D2969000321218BF754F
:0B1EC60082071219C2758207121A5120
:081ED100200807E54B60030245
:021ED9002020C7
:091EDB00C20820130675820012F2
:021EE4001AAB37
:0C1EE600D20A7582191219237496C0E00C
:0E1EF2007401C0E0907A6775F08012171C151D
:0E1F00008115819002BC1218BF7496C0E07467
:0E1F0E0001C0E0907A7075F08012171C1581EA
:041F1C0015817A00B1
:031F2000BA040000
:0E1F2300502FC296D296758201C002121A7615
:0E1F3100D002900096C0021218BFD002758236
:0E1F3F0000C002121A76D002900096C0021264
:071F4D0018BFD0020A80CC8E
:0E1F540074C8C0E0E4C0E0907A5575F08012C9
:0A1F6200171C158115811260901202
:091F6C002120758207121A51753B
:051F75004304022020DE
:071F7A00E546600302202090
:091F8100D20A75430175820412B5
:0E1F8A0019C27496C0E07401C0E0907A6775C9
:0D1F9800F08012171C1581158190012C128C
:0E1FA50018BFC296D2967496C0E07401C0E0D8
:0E1FB300907A7975F08012171C1581158190B7
:0E1FC100012C1218BF7496C0E07401C0E090AD
:0E1FCF007A8275F08012171C158115817582BB
:041FDD0003121A5180
:0E1FE100121A5AE582701B758207122057747F
:0C1FEF00205532F582121A769000011283
:081FFB0018BFC296D29680DEE9
:0E2003007407C0E075822112155F1581758289
:0C20110001121A76758207121A51800322
:03201D0075430008
:0A202000E5345401FAE4A21B33FB7F
:05202A00B50202802256
:06202F00E53413921BE5ED
:072035004B24FF5002154B84
:0C203C00C374808546F063F08095F0507E
:0720480008E534600280028C
:02204F00154634
:06205100855981D05922DF
:0A205700AA8274F925495003754967
:01206100007E
:09206200E532C3954AFBBB050001
:03206B00500122FF
:04206E0085324AE588
:0B20720049907A8B93FBC0028B821216
:07207D00155F1581054922E2
:0A208400AA8274FA25495003754939
:01208E000051
:09208F00E532C3954AFBBB0800D1
:03209800500122D2
:04209B0085324AE55B
:0B209F0049907A9293FBC0028B8212E2
:0720AA00155F1581054922B5
:0A20B100AA8274FC2549500375490A
:0120BB000024
:0920BC00E532C3954AFBBB0C00A0
:0320C500500122A5
:0420C80085324AE52E
:0B20CC0049907A9893FBC0028B8212AF
:0720D700155F158105492288
:0A20DE00AA8274F4254950037549E5
:0120E80000F7
:0920E900E532C3954AFBBB0C0073
:0320F20050012278
:0420F50085324AE501
:0C20F90049907A9C93FBC002C0028B82CD
:0B21050012155F1581D0020AE5499019
:0E2110007AA893FBC0028B8212155F15810521
:02211E00492254
:0921200012609074022535FA8565
:072129003382C002C0341232
:0E21300063E4158115811264DFAA82AB83ACD3
:0E213E00F01273C9FA7408C0E0E4C0E08A82AF
:0E214C0012160C158115811264DFAA82AB8376
:0E215A00ACF074042AFAE43BFB8A828B838C7F
:0E216800F01273C9FA7408C0E07404C0E08A73
:0E2176008212160C158115811264DFAA82AB4D
:0E21840083ACF074022AFAE43BFB8A828B8360
:0E2192008CF01273C9FA7409C0E07402C0E048
:0E21A0008A8212160C158115811264DFAA8244
:0921AE00AB83ACF00ABA00010B8E
:0E21B7008A828B838CF01273C9FA7408C0E020
:0E21C5007401C0E08A8212160C158115811279
:0E21D30064DFAA82AB83ACF074032AFAE43B0B
:0E21E100FB8A828B838CF01273C9FA7408C0DB
:0E21EF00E07403C0E08A8212160C158115817F
:0E21FD001264DFAA82AB83ACF074052AFAE408
:0E220B003BFB8A828B838CF01273C9FA740835
:0E221900C0E07405C0E08A8212160C15811513
:0E222700811264DFAA82AB83ACF074062AFA3F
:0E223500E43BFB8A828B838CF01273C9FA742F
:0E22430007C0E07406C0E08A8212160C1581F6
:0E22510015811264DFAA82AB83ACF074072AF9
:0E225F00FAE43BFB8A828B838CF01273C9FA7F
:0E226D007402C0E07407C0E08A8212160C15DD
:04227B008115812226
:0A227F00E5315401FAE4A21C33FB20
:0B228900B50242E5315401FAB4010037
:07229400921C100E02800CE9
:0A229B0090003375F04012286785AB
:0222A500314CBA
:0A22A700E531C3954CFA2421501DC7
:0422B10085314C9097
:0D22B500003375F040122A05E582700D120D
:0A22C2002849E5827006121AC012C6
:0222CC00377168
:0A22CE0030032A90003375F040122F
:0C22D8006A11AA82BA0057D310AF01C3EC
:0922E400C0D0E533FA14F533C251
:0C22ED0003D0D092AF90003375F0400297
:0222F900286754
:0E22FB0090003375F040126A11AA82BA0202F6
:02230900800E44
:0E230B0090003375F040126A11AA82BA011DCB
:05231900D310AF01C369
:0A231E00C0D0AA3374012AF533D2AF
:0C23280003D0D092AF90003375F040025B
:02233400286718
:012336002284
:0A23370030140D90003675F04012CE
:062341006B65AA82800218
:022347007A001A
:072349002010042014012202
:05235000E4BA000104E5
:08235500FB7008BA01028003CD
:03235D000224B2A5
:0C236000C002C003126090D003D0022025
:03236C001001223B
:0E236F0090003675F040C002C0031265A9ACA4
:0D237D0082D003D002EC24F850030224307B
:07238A00EC2C2C9023917351
:072391000224300223A9021F
:0623980023BD0223D10267
:06239E0023E40223F70214
:0523A400240A02241DC3
:0E23A900907AB475F080C002C0031260B5D007
:0623B70003D002022441E4
:0E23BD00907ABD75F080C002C0031260B5D0EA
:0623CB0003D002022441D0
:0E23D100907AC675F080C002C0031260B5D0CD
:0523DF0003D002805D47
:0E23E400907ACF75F080C002C0031260B5D0B1
:0523F20003D002804A47
:0E23F700907AD875F080C002C0031260B5D095
:0524050003D002803746
:0E240A00907AE175F080C002C0031260B5D078
:0524180003D002802446
:0E241D00907AEA75F080C002C0031260B5D05C
:05242B0003D002801146
:0E243000907AF375F080C002C0031260B5D040
:03243E0003D002C6
:0E244100C002C0031264DFAC82AD83AEF0D0E7
:0E244F0003D002C002C00374DCC0E07401C000
:0E245D00E08C828D838EF012171C1581158184
:06246B00D003D0027C004A
:03247100BC230089
:0E247400503C900019C002C003C0041218BFF3
:0D248200D004D003D002C002C003C0041279
:0E248F001B27D004D003D002C002C003C0043B
:0C249D00121B4AD004D003D002E53960C5
:0224A90001220E
:0724AB00C296D2960C80BF1F
:0624B20020100302256169
:0C24B800C002C003126090D003D0028567
:0C24C4003682C002C0031262B3D003D005
:0E24D00002907AFC75F080C002C0031260B565
:0C24DE00D003D002853782C002C0031278
:0E24EA006337D003D002C002C0031264DFAC1F
:0E24F80082AD83AEF0D003D002C002C00374E8
:0E250600DCC0E07401C0E08C828D838EF01288
:0C251400171C15811581D003D0027C003B
:03252000BC3200CA
:0E252300503C900019C002C003C0041218BF43
:0D253100D004D003D002C002C003C00412C9
:0E253E001B27D004D003D002C002C003C0048B
:0C254C00121B4AD004D003D002E5396015
:0225580001225E
:07255A00C296D2960C80BF6F
:08256100EB7044BA0102803F57
:0E2569008A82127198AA82AB837C808A828B50
:08257700838CF012275A7A0050
:03257F00BA280077
:0E2582005024900019C0021218BFD002C002EF
:0D259000121B27D002C002121B4AD002E528
:04259D00396001227E
:0725A100C296D2960A80D712
:0725A800126090853382C030
:0425AF0035C03412ED
:0C25B30063E415811581C37438954074F1
:0C25BF00049541500F7582031260EA90F1
:0825CB007AFF75F0801260B583
:0E25D3001264DFAA82AB83ACF074DCC0E0E4DB
:0E25E100C0E08A828B838CF012171C158115C6
:0225EF00812247
:0825F100C059858159058120C4
:0525F90011030226E5BC
:0C25FE00126090AA590A7B007C408A827F
:0C260A008B838CF0122E32E582602CA82D
:0B2616005908C3E664809477500B90D5
:0A2621007B0375F0801260B580099C
:09262B00907AFF75F0801260B591
:09263400A85908A8590886821271
:04263D00622380098B
:09264100907B0675F0801260B573
:0A264A00907B0C75F0801260B51251
:0E26540064DFAA82AB83ACF074DCC0E0E4C0AB
:0E266200E08A828B838CF012171C1581158183
:022670007A00EE
:03267200BA50005B
:0E2675005025900019C0021218BFD002C002FA
:0D268300121B27D002C002121B4AD002E534
:052690003960028050DA
:07269500C296D2960A80D61E
:07269C00126090853382C03B
:0426A30035C03412F8
:0C26A70063E415811581C37438954074FC
:0C26B300049541500F7582031260EA90FC
:0826BF007AFF75F0801260B58E
:0E26C7001264DFAA82AB83ACF074DCC0E07456
:0E26D50001C0E08A828B838CF012171C1581E5
:0226E30015815F
:0626E500855981D0592245
:0A26EB00E5315401FAE4A21D33FBAF
:0B26F500B50244E5315401FAB40100C5
:09270000921D126090C37438951B
:08270900407404954150128553
:09271100338274FFC0E0C03412F1
:08271A0063E415811581800EB6
:06272200853382C035C0C2
:08272800341263E415811581F0
:0C2730001264DFAA82AB83ACF01216D258
:0A273C00C3743895407404954150B1
:0E274600127405C0E075822012155F158175B2
:0527540082060220DEF8
:01275900225D
:0D275A00AA82AB83ACF0C002C003C0041221
:0A2767006090D004D003D0027D0082
:0E277100ED2AFEE43BFF8C008E828F8388F001
:0A277F001273C9FEBE0003022821F8
:03278900BDFF0091
:05278C004003022821BA
:0E279100C296D296BE0A6C907A5575F080C042
:0E279F0002C003C004C0051260B5D005D0040E
:0D27AD00D003D002C002C003C004C005125A
:0E27BA0064DFAF82A883A9F0D005D004D0035D
:0E27C800D002C002C003C004C0057482C0E08D
:0E27D6007401C0E08F82888389F012171C15F1
:0E27E400811581D005D004D003D002C002C000
:0E27F20003C004C005126090D005D004D003CF
:04280000D00280156D
:0E2804008E82C002C003C004C00512609BD0CB
:0728120005D004D003D00241
:082819000DC296D29602277150
:0A282100907A5575F0801260B51230
:0E282B0064DFAA82AB83ACF07482C0E074015B
:0E283900C0E08A828B838CF012171C1581156B
:022847008122EC
:0D284900758268123803E5827003F5822263
:0D28560075820012384EE5827003F5822273
:042863007582012257
:0E286700AA82AB83ACF0BA0009BB0006BC002D
:0428750003022849E9
:0E287900758268C002C003C004123803E582F5
:0B288700D004D003D0027003F58222C1
:0E289200758200C002C003C00412383AD004A0
:0928A000D003D002D310AF01C334
:0E28A900C0D074022AFDE43BFE8C078D828EA7
:0E28B700838FF01273C9FD75F00A84FEC454BD
:0E28C500F0FE75F00AED84E5F0FD2EF582C000
:0E28D30002C003C00412383AD004D003D00271
:0E28E10074012AFDE43BFE8C078D828E838FEE
:0E28EF00F01273C9FD75F00A84FEC454F0FEA9
:0E28FD0075F00AED84E5F0FD2EF582C002C0F4
:0E290B0003C00412383AD004D003D0028A82EE
:0E2919008B838CF01273C9FD75F00A84FEC426
:0E29270054F0FE75F00AED84E5F0FD2EF58209
:0E293500C002C003C00412383AD004D003D050
:0E29430002758200C002C003C00412383AD0F0
:0E29510004D003D00274032AFDE43BFE8C0781
:0E295F008D828E838FF01273C9FD75F00A848D
:0E296D00FEC454F0FE75F00AED84E5F0FD2E78
:0E297B00F582C002C003C00412383AD004D066
:0E29890003D00274032AFAE43BFB74012AFD1A
:0E299700E43BFE8C078D828E838FF01273C995
:0E29A500FD75F00A84FEC454F0FE75F00AEDD4
:0E29B30084E5F0FD2EF582C002C003C00412C0
:0E29C100383AD004D003D00274022AFAE43B64
:0E29CF00FB8A828B838CF01273C9FA75F06458
:0E29DD0084E5F075F00A84FBC454F0FB75F03D
:0E29EB000AEA84E5F0FA2BF58212383AD0D0D1
:0C29F90092AF75821012384E75820122D8
:0A2A0500C059858159C082C083C00A
:0C2A0F00F0E581240DF581A85908B600FF
:0D2A1B000E08B6000A08B60006122849028F
:022A28002D1867
:0D2A2A00758268123803E5827005F582029E
:022A37002D1858
:0E2A390075820012384E7582681237A0E58251
:072A47007005F582022D1855
:0C2A4E001237DBAD82E559240AF8A6051A
:0A2A5A00E55924042402F8E559248C
:0E2A64000AF9E7C4540FFE740F5E75F00AA461
:0C2A7200FFE559240AF9740F572FA6E065
:0B2A7E00E559240AF9E730E70276FF73
:0C2A8900740F5E75F00AA4FEE559240AE3
:0D2A9500F9740F572EA6E01237DBAE82E574
:0A2AA20059240AF8A606E559240499
:0C2AAC002401F8E559240AF9E7C4540F8E
:0C2AB800FE740F5E75F00AA4FEE55924C0
:0E2AC4000AF9740F572EA6E01237DBAE82E53A
:0A2AD20059240AF8A606E559240469
:0C2ADC00F8E559240AF9E7C4540FFE7411
:0C2AE8000F5E75F00AA4FEE559240AF9FF
:0E2AF400740F572EA6E01237DB1237DBAE82CE
:0A2B0200E559240AF8A606E5592457
:0C2B0C00042403F8E559240AF9E7C45436
:0C2B18000FFE740F5E75F00AA4FEE55974
:0E2B2400240AF9740F572EA6E01237DBAE829A
:0A2B3200E559240AF8A606E5592427
:0C2B3C000424032401F8E559240AF9E7F9
:0D2B4800C4540FFE740F5E75F00AA4FEE584
:0B2B550059240AF9740F572EA6E01255
:0C2B600037E8AE82E559240AF8A606E525
:0B2B6C00592404FE74032E2402F8E537
:0C2B770059240AF9E7C4540FFF740F5FE3
:0C2B830075F00AA4FFE559240AF9740F4C
:0E2B8F00572FA6E074022EF88606EE24C450DE
:072B9D0006758200022D18ED
:0C2BA400E5592404F8740128F98706EEB6
:0A2BB00024C45006758200022D189F
:0D2BBA008606EE24E85006758200022D18F4
:0C2BC700E55924042403FE74022EF88655
:0E2BD3000774012EF88682C00712654FAE828D
:0A2BE1001581E559240AF8A606E55F
:0B2BEB0059240AF8B6FF0675820002AC
:022BF6002D1898
:0C2BF800E5592404FE74032EF88607BF84
:022C04000100CD
:0C2C0600400AE559240AF8C3E69F500676
:062C1200758200022D187E
:0E2C18007F007A408E828F838AF0126A11AAA2
:062C260082E4BA01010482
:0B2C2C006009E559240AF876018007D2
:072C3700E559240AF87600BC
:052C3E00D310AF01C33B
:0A2C4300C0D0E5592404F88606A964
:0C2C4D00590987820987830987F0EE127D
:0C2C590073B0A95909740127FEE4093783
:0E2C6500FF098705740128F987028E828F838C
:0C2C73008DF0EA1273B0A9590974022711
:0E2C7F00FAE40937FB098704080886058A82F3
:0C2C8D008B838CF0ED1273B0A859087412
:0C2C99000326FAE40836FB088604E5591F
:0E2CA5002404FD74032DF886068A828B838C2E
:0C2CB300F0EE1273B0A85908740326FA62
:0C2CBF00E40836FB088604E559240BF8F5
:0E2CCB0074012AF6E43B08F608A6040D0D0D70
:0C2CD90074012DF88606E559240BF886DE
:0E2CE500820886830886F0EE1273B074022A0D
:0E2CF300FAE43BFB74022DF886058A828B837F
:0C2D01008CF0ED1273B0E559240AF8E6DE
:0B2D0D0024FF9203D0D092AF7582012A
:062D1800855981D059220B
:0B2D1E00758268123803E58270012204
:0E2D290075820012383A75828012383A75822F
:0E2D37000012383A75820012383A7582001286
:0C2D4500383A75820112383A758201128A
:0C2D5100383A75820112383A758210027F
:022D5D00384EEE
:0A2D5F00C059858159E582FA24C8A5
:072D69005005758200805344
:0E2D7000758268C002123803E582D00270043A
:042D7E00F582804119
:0E2D820074082AF58212384E7582681237A046
:082D9000E5827004F582802B3E
:0C2D9800E55924FBF88602088603088633
:0E2DA40004C002C003C0041237E8AD82D004A0
:0E2DB200D003D0028A828B838CF0ED1273B0B6
:032DC00075820118
:062DC300855981D0592260
:0A2DC900C059858159E582FA24C83B
:072DD30050057582008034F9
:0E2DDA00758268C002123803E582D0027004D0
:042DE800F5828022CE
:0C2DEC0074082AF58212383AA859181809
:0C2DF80018A859181818868212384EE5E9
:072E0400827004F5828003D7
:032E0B00758201CC
:062E0E00855981D0592214
:0D2E140075824F123803E5827003F58222AB
:0D2E210075820012384EE5827003F58222A2
:042E2E007582012286
:0E2E3200AA82AB83ACF0BA0009BB0006BC005C
:042E400003022E1447
:092E4400E531C3954EFDBD03000C
:0C2E4D00501AAD4D8A828B838CF0ED1280
:072E590073B0E4BD80010429
:042E6000FDB40100BC
:052E6400E433F58222B9
:0A2E690085314E8A828B838CF07451
:0E2E7300801273B075824FC002C003C00412FB
:0E2E810037A0E582D004D003D002602AC00240
:0E2E8F00C003C0041237DBAD82D004D003D0E4
:0E2E9D00028A828B838CF0ED1273B0C002C0EB
:0C2EAB0003C0041237E8D004D003D002AA
:0E2EB7008A828B838CF01273C9FDC3648094F1
:0E2EC5004E40168A828B838CF01273C9FDC3B7
:0B2ED30074B28DF063F08095F0500B9E
:0B2EDE008A828B838CF074801273B02A
:0C2EE9008A828B838CF01273C9FA8A4D28
:052EF500E4BA800104B5
:042EFA00FAB4010025
:052EFE00E433F582221F
:0A2F0300C059858159C082C083C007
:0E2F0D00F0758201121A76758203121A51E5D0
:0C2F1B005924FBF8860508860608860786
:082F2700AA39BA00030231D2FD
:052F2F007539008A0461
:0D2F3400C374808CF063F08095F0400302C0
:022F41003067F7
:0C2F4300C005C006C007A8590886820817
:0C2F4F0086830886F01273C9FDBD5A008D
:0C2F5B00D007D006D005401DA8590886FC
:0E2F6700820886830886F0745A1273B08D8239
:0B2F75008E838FF0E41273B00230670F
:0C2F8000C005C006C007A85908868208DA
:0E2F8C0086830886F01273C9FDC3741D9DE490
:0C2F9A0033D007D006D0056037A85908D6
:0E2FA60086820886830886F01273C9FA75F0D9
:0C2FB4000584ABF07405C39B2AFAA859F1
:0E2FC0000886820886830886F0EA1273B08DB8
:0C2FCE00828E838FF0E41273B002305D3D
:0C2FDA00A8590886820886830886F01239
:0C2FE60073C9FA24F6502BA85908868203
:0C2FF2000886830886F01273C904FAA850
:0C2FFE00590886820886830886F0EA12D3
:0E300A0073B08D828E838FF0E41273B0804518
:0D3018008D828E838FF01273C9FABA1E00EC
:0D302500402B8D828E838FF0E41273B0A8D3
:0B303200590886820886830886F01289
:0C303D0073C904FAA8590886820886832B
:093049000886F0EA1273B0800B56
:0B3052008D828E838FF0741E1273B00D
:0A305D001C8C02C296D296022F349A
:07306700EA20E7030231C07B
:0C306E00A8590886820886830886F012A4
:0C307A0073C9FB24E15071A8590886823C
:0E3086000886830886F01273C9FB75F0058476
:07309400ABF0BB0002802A33
:0C309B00A8590886820886830886F01277
:0E30A70073C9FB75F00584ACF07405C39C2B57
:0C30B500FBA8590886820886830886F074
:0430C100EB1273B0EB
:0C30C500A8590886820886830886F0124D
:0C30D10073C924FBFBA8590886820886FE
:0E30DD00830886F0EB1273B08D828E838FF025
:0730EB00E41273B00231B8DA
:0C30F200A8590886820886830886F01220
:0E30FE0073C9FB24F550458D828E838FF0122E
:0E310C0073C9FB24FF500C8D828E838FF0E47C
:05311A001273B0801FDC
:0C311F00A8590886820886830886F012F2
:0C312B0073C9FB1BA85908868208868324
:073137000886F0EB1273B0F3
:0C313E008D828E838FF0E41273B0806EDF
:0D314A008D828E838FF01273C9FB703DA83B
:0B315700590886820886830886F01263
:0E31620073C9FB60598D828E838FF0741E122C
:0C31700073B0A859088682088683088680
:0C317C00F01273C9FB1BA85908868208DA
:0B31880086830886F0EB1273B08025F0
:0E3193008D828E838FF01273C9FB24E1500DE4
:0D31A1008D828E838FF0741E1273B0800A31
:0A31AE008D828E838FF0E41273B05F
:0831B8000AC296D296023067AC
:0E31C000758202C005C006C007121A51D00762
:0431CE00D006D00552
:0E31D200C005C006C007126090D007D006D01E
:0E31E00005907B1175F080C005C006C0071277
:0C31EE0060B5D007D006D005A8590886AF
:0E31FA00820886830886F01273C9FAF582C037
:0E32080005C006C0071262F5D007D006D0053B
:0E32160075823AC005C006C00712609BD00743
:0E322400D006D0058D828E838FF01273C9FA0A
:0E323200F582C005C006C007126282D007D028
:0D32400006D005758220C005C006C007122B
:0E324D00609BD007D006D005C005C006C007A4
:0E325B001264DFAA82AB83ACF0D007D006D09D
:0E326900058A828B838CF0C005C006C0071258
:0C32770016D2D007D006D005A859088652
:0E328300820886830886F01273C9FABA0A0020
:0E329100502BC005C006C007E4C0E0758220C7
:0E329F0012155F1581D007D006D0057582018B
:0E32AD00C005C006C007122084D007D006D08E
:0332BB0005802A61
:0E32BE00758200C005C006C007122084D0072C
:0E32CC00D006D005C005C006C0077401C0E0E2
:0E32DA0075822012155F1581D007D006D00531
:0E32E800C296D296C005C006C007121A5AE55B
:0C32F60082D007D006D0057003022F27FD
:0C330200A8590886820886830886F0120D
:0E330E0073C9FA706E8D828E838FF01273C9B0
:0E331C00FA7062907B1475F080C005C006C088
:0E332A00071216D2D007D006D005758219C042
:0E33380005C006C007121923D007D006D00525
:0E334600758200C005C006C007121A76D007B7
:0E335400D006D005C296D2969003E8C005C000
:0E33620006C0071218BFD007D006D0058D8216
:0E3370008E838FF0741E1273B0121B1D7582B7
:03337E000080507C
:0C338100A8590886820886830886F0128E
:0E338D0073C9FAC005C006C007C002758207EA
:0E339B00122DC91581D007D006D0058D828E67
:0D33A900838FF01273C9FDC00575820812F4
:0E33B6002DC91581758207121A517582FF12FA
:0833C4001A76C208758201129D
:0533CC0019C275820129
:0633D100855981D059224C
:0A33D700C059858159C082C083C02F
:0C33E100F00581A8590886820886830840
:0C33ED0086F01273C9FDE5592404F8A60F
:0C33F90005E55924FBF886060886070845
:0E34050086058E828F838DF01273C9FAC00285
:0E341300C005C006C0071214F1D007D006D0C5
:0B34210005D002E5592404F8B60A00AB
:0E342C005024C002C005C006C0077404C0E0F2
:0E343A007401C0E075820412160C1581158114
:0A344800D007D006D005D002802185
:0E345200C002C005C006C0077404C0E0E4C09C
:0E346000E075820412160C15811581D007D07C
:05346E0006D005D002AC
:0A347300C20875390075821EC00200
:0E347D00C005C006C007121A51D007D006D0F5
:07348B0005D002C296D296A3
:08349200AB39BB000302352A2F
:03349A0075390081
:0E349D00C374808BF063F08095F0502F75F0B3
:0E34AB0005EA84ACF07405C39CFC2AFABA3C16
:0134B9000012
:0B34BA0040197A00E5592404F806E5EB
:0734C500592404F8B61800B9
:0934CC004007E5592404F87600DC
:0334D5001B80C594
:0E34D800EB30E73475F005EA84ACF0BC00027E
:0234E60080075D
:0734E8007405C39CFC2AFAE5
:0C34EF00BA0017E5592404F8B60007E500
:0634FB00592404F87618C4
:08350100E5592404F8167A3C98
:07350900EA24FBFA0B80C865
:0E35100075821EC002C005C006C007121A5107
:0C351E00D007D006D005D002C296D2968D
:0E352A00C006C007C005C002C005C006C0072D
:0E353800126090D007D006D005D002907B1113
:0E35460075F080C002C005C006C0071260B557
:0E355400D007D006D005D002C002C005C006C8
:0C356200C00774FFC0E0C002E55924045B
:0C356E00F8E5592404F886821263E41585
:0E357A00811581D007D006D005D002758220C1
:0E358800C002C005C006C00712609BD007D06D
:0E35960006D005D002C002C006C0071264DFD6
:0E35A400AB82AC83ADF0D007D006D0028B8294
:0D35B2008C838DF0C002C005C006C007125A
:0C35BF0016D2D007D006D005D002E55986
:0635CB002404F8B60A001A
:0E35D100E433D005D007D0066033C002C00539
:0E35DF00C006C007E4C0E075822012155F151B
:0E35ED0081D007D006D005D002758201C00241
:0E35FB00C005C006C007122084D007D006D03D
:0536090005D002803233
:0E360E00758200C002C005C006C007122084ED
:0E361C00D007D006D005D002C002C005C006FF
:0E362A00C0077401C0E075822012155F158183
:08363800D007D006D005D00236
:0D364000C296D296C002C005C006C0071297
:0E364D001A5AE582D007D006D005D0026025BB
:0D365B00907B1475F0801216D27582191242
:0E3668001923C296D2969003E81218BFC2969C
:0A367600D296121B1D7582008036EB
:0636800020080302349251
:0C368600A8590886820886830886F0E5B3
:0C369200592404F9E71273B08E828F8374
:0E369E008DF0EA1273B075820812192375823E
:0A36AC00081219C2121B1D758201DD
:0636B600855981D0592264
:097A2800D7205254432020200015
:097A31005765636B656E203F0090
:097A3A00526164696F20202000F4
:097A43006CE4756674202020003B
:097A4C00626572656974732E0015
:097A550020202020202020200028
:097A5E005765636B65722120007D
:097A67005765636B65721620007F
:097A70002020617573162020002E
:097A790016776965646572160058
:097A820016616B74697620200086
:077A8B0093949596979899DA
:067A9200040506070605CD
:047A9800131415149A
:0C7A9C002020207F808182838281807FF7
:0C7AA800202020848586878887868584BE
:097AB4004D6F6E74616720200023
:097ABD004469656E737461670091
:097AC6004D697474776F63680068
:097ACF00446F6E6E6572732E00A7
:097AD800467265697461672000C3
:097AE10053616D737461672000AC
:097AEA00536F6E6E746167200099
:097AF30020203F3F3F3F2020000E
:037AFC000B20005C
:047AFF002020200023
:037B03002020003F
:067B06002020202D2D00BF
:057B0C00B04320200041
:037B11000909005F
:097B1400202020D73AD7D7200029
:0200D600C21E48
:0236BC007A0092
:0836BE000ABA00047582002223
:0B36C6000000003095F210940280ED2F
:0236D1007A0578
:0E36D300000000DAFBC29500000075820122A3
:0936E100C295C294000000D295CC
:0536EA003095FD7A059A
:0736EF00000000DAFBD29499
:0736F6003094FD00000022EA
:0436FD00AA827B0022
:03370100BB080002
:0C3704005018EA2A9294FA000000D295B6
:0E3710003095FD000000000000C2950B80E324
:04371E00D294D295DA
:0E3722003095FD000000309406C295758200BF
:013730002276
:06373100C2957582012221
:06373700AA827B007C0861
:0A373D00EC24FF501AEB2BFBD29591
:0E3747003095FDE4A29433FD4203000000C261
:07375500950000001C80E15B
:04375C00EAB40100CA
:043760009294D295D8
:0D3764003095FD000000C295D2948B8222AA
:0C377100C21EC295C2940000001236E196
:02377D007A00D0
:03377F00BA80000D
:0E378200500DC295000000D2950000000A8094
:01379000EE4A
:06379100309503209404B2
:043797007A00800232
:02379B007A01B1
:03379D008A8222FB
:0A37A000E582FA30E704758200228A
:0737AA00301E0475820022AD
:0E37B100C0021236BCE582D0027003F58222FF
:0E37BF00EA2AFA74014AF5821236FDE582709C
:0837CD00071236E175820022AB
:0637D500D21E75820122E4
:0737DB00201E0475822A2262
:0637E20075820102373779
:0C37E8007A2A301E13758200123737ABAE
:0C37F400828B02C0021236E1D002C21E1D
:033800008A822297
:0A380300E582FA30E7047582002226
:07380D00301E047582002249
:0E381400C0021236BCE582D0027003F582229B
:0E382200EA2AF5821236FDE58270071236E1C1
:04383000758200227B
:06383400D21E7582012284
:0C383A00AA82301E0E8A821236FDE58242
:0738460070051236E1C21EFD
:01384D002258
:09384E00AA82201E0475820022EA
:0C3857008A821236FDE58224FF921EE5F5
:093863008224FF921E1236E120BE
:06386C001E04758200221B
:06387200C21E7582012256
:0700D800751B00751C00758B
:0A00DF001D00C220E4A2B03325E0AA
:0900E900FAE4A2B133FB4AF51F51
:0E387800C2AF5389F0438901758C00758A0137
:0E388600D2A9C28DD28C53890F438910758D43
:0E38940000758B01D2ABC28FD28E75B800D2F8
:0938A200BBD2AF9000140218BF64
:0E38AB00C0E0C0F0C082C083C002C003C004F1
:0C38B900C005C006C007C000C001C0254B
:0E38C500C0D075D008C2AF758CEC7478258A1F
:0C38D3002402F58AD2AF309104C20480B8
:0138DF001BCD
:0838E00030040FE5196014E546
:0638E80019B40102D20632
:0438EE00151980091F
:0538F200D204D20575AF
:0438F70019FAD20ADE
:0738FB0030B204C207801B7C
:0839020030070FE51A6014E51F
:06390A001AB40102D2090B
:04391000151A8009FB
:05391400D207D2087586
:043919001AFAD20ABA
:0A391D00301525E53230E61C75D0A8
:0C392700001214EA75D008AA82BA04004D
:083933005006D2B3C2B4800AB1
:06393B00C2B3D2B4800407
:04394100D2B3D2B477
:0739450005180532749C25F2
:06394C0018503E05317524
:0C395200180090003375F04075D0001292
:0B395E00687B75D008E535600280240E
:0A396900AA40AB417C007D00C3EAD8
:0E39730094FEEB94FFEC9400ED648094805081
:093981000B74012540F540E4350A
:03398A0041F541C3
:07398D00309304051B8002CA
:02399400151B01
:0A399600C3E51B6480947D500375A7
:0239A0001BFD0D
:0C39A200C37483851BF063F08095F05027
:0439AE0003751B037F
:0939B200E51B30E704C228800285
:0239BB00D22810
:0939BD00051DE51C24F65003026F
:0239C6003AF3D2
:0539C800E51C251C2593
:0539CD001C9039D273CB
:0739D2000239F0023A07027E
:0639D9003A27023A3E020B
:0639DF003A51023A6F02AA
:0639E5003A86023A9D0241
:0539EB003ABA023AD7D0
:0839F000E51DB4F007D20D75CE
:0439F8001D00800628
:0639FC00202803751C01E8
:053A0200C20F023E4D61
:083A0700E51DB4F00CD20D75B1
:063A0F001D00751C00C241
:033A15000F800C13
:073A1800302809751D00753F
:053A1F003C00751C02D3
:033A2400023E4D12
:063A2700202809D20D75F4
:063A2D001C01C20F80081D
:083A3300E51DB40603751C0338
:033A3B00023E4DFB
:083A3E00202805751C04800816
:083A4600E51DB40E03751C051B
:033A4E00023E4DE8
:063A5100302809D20D75BA
:063A57001C00C20F800FED
:093A5D00E51DB45A0A751C08C2EB
:043A660029B20C0273
:023A6A003AFC24
:033A6C00023E4DCA
:063A6F00202809D20D75AC
:063A75001C01C20F8008D5
:083A7B00E51DB41003751C06E3
:033A8300023E4DB3
:083A8600202805751C07800CC7
:083A8E00E51DB41807D20DC2BA
:043A96000F751C008C
:033A9A00023E4D9C
:063A9D00302809D20DC221
:063AA3000F751C00800EEF
:093AA900E51DB45A09751C08D290
:053AB20029B20C804563
:033AB700023E4D7F
:073ABA0030280F751D00AA62
:073AC1003C74012AF53C757D
:043AC8001C02800854
:083ACC00E51DB49603751C0909
:033AD400023E4D62
:063AD70030280CD20D7531
:063ADD001D00751C00C273
:033AE3000F800A47
:093AE600E51DB4B405751C01B224
:013AEF000BCB
:033AF000023E4D46
:073AF300751D00751C0002A7
:023AFA003E4D3F
:0A3AFC00C3E53C94115003023E4D57
:053B0600302902B21F8E
:053B0B00AA3CBA110004
:053B10005003023DEE30
:083B1500EA24C55003023DEE55
:0E3B1D00EA24EFFA240983C0E0EA242D83C0D5
:023B2B00E02296
:023B2D0081888D
:023B2F009C9F59
:023B3100A8B535
:023B3300BFCB06
:023B3500D7E3D4
:023B3700EFFBA2
:023B39002C3925
:023B3B00434FF6
:023B3D005B67C4
:023B3F0073927F
:023B41009FA93A
:023B4300B5C10A
:023B4500CDF6BB
:023B4700FF0974
:023B4900222B2D
:023B4B00354102
:023B4D004D76B3
:023B4F007F896C
:023B510095A13C
:023B5300ADB90A
:023B5500C5E9C0
:023B57003B3BF6
:023B59003B3BF4
:023B5B003B3BF2
:023B5D003B3BF0
:023B5F003B3BEE
:023B61003B3BEC
:023B63003C3CE8
:023B65003C3CE6
:023B67003C3CE4
:023B69003C3CE2
:023B6B003C3CE0
:023B6D003C3CDE
:023B6F003C3CDC
:023B71003C3DD9
:023B73003D3DD6
:023B75003D3DD4
:023B77003D3DD2
:023B79003D3DD0
:023B7B003D3DCE
:023B7D003D3DCC
:023B7F003D3DCA
:053B8100A229922002C0
:023B86003E4DB2
:0A3B8800E4A22933FAE4A22033FB83
:073B9200EAB50B03753C00CE
:033B9900023E4D9C
:033B9C00023E4D99
:063B9F00202903753C0023
:033BA500023E4D90
:063BA800A229921FE4A215
:053BAE002933F51E02A1
:023BB3003E4D85
:063BB500302904051E0585
:013BBB001EEB
:033BBC00023E4D79
:083BBF00302906E51E2404F57F
:013BC7001EDF
:033BC800023E4D6D
:083BCB003029067408251EF5DF
:013BD3001ED3
:033BD400023E4D61
:083BD700302906740A251EF5D1
:013BDF001EC7
:033BE000023E4D55
:083BE3003029067414251EF5BB
:013BEB001EBB
:033BEC00023E4D49
:083BEF003029067428251EF59B
:013BF7001EAF
:033BF800023E4D3D
:063BFB00151E201F06E567
:053C01001E24C4500365
:033C0600753C000A
:0A3C0900300F1AAA1E7B001ABAFF42
:023C1300011B93
:0C3C1500AC3B7D00ECB50A06EDB50B02DF
:023C210080031E
:033C2300753C00ED
:043C2600851E3B02BA
:023C2A003E4D0D
:063C2C00A229921FE4A290
:053C32002933F51E021C
:023C37003E4D00
:063C3900302904051E0500
:013C3F001E66
:033C4000023E4DF4
:083C4300302906E51E2404F5FA
:013C4B001E5A
:033C4C00023E4DE8
:083C4F003029067408251EF55A
:013C57001E4E
:033C5800023E4DDC
:083C5B00302906740A251EF54C
:013C63001E42
:033C6400023E4DD0
:083C67003029067414251EF536
:013C6F001E36
:033C7000023E4DC4
:093C7300201F06E51E24E85003A1
:033C7C00753C0094
:063C7F00300F0AE53AB522
:043C85001E02800398
:033C8900753C0087
:043C8C00851E3A0255
:023C90003E4DA7
:063C9200A229921FE4A22A
:053C98002933F51E02B6
:023C9D003E4D9A
:063C9F00302904051E059A
:013CA5001E00
:033CA600023E4D8E
:083CA900302906E51E2404F594
:013CB1001EF4
:033CB200023E4D82
:083CB5003029067408251EF5F4
:013CBD001EE8
:033CBE00023E4D76
:083CC100302906740A251EF5E6
:013CC9001EDC
:033CCA00023E4D6A
:083CCD003029067414251EF5D0
:013CD5001ED0
:0A3CD600E51E6006E51E24E0500321
:033CE000753C0030
:063CE300300F0AE53DB5BB
:043CE9001E02800334
:033CED00753C0023
:043CF000851E3D02EE
:023CF4003E4D43
:073CF600E4A22933F51E02D0
:023CFD003E4D3A
:063CFF00302904051E053A
:013D05001E9F
:033D0600023E4D2D
:083D0900302906E51E2404F533
:013D11001E93
:0A3D1200E51E6006E51E24F85003CC
:033D1C00753C00F3
:033D1F00023E4D14
:073D2200E4A22933F51E02A3
:023D29003E4D0D
:063D2B00302904051E050D
:013D31001E73
:033D3200023E4D01
:083D3500302906E51E2404F507
:013D3D001E67
:033D3E00023E4DF5
:083D41003029067408251EF567
:013D49001E5B
:033D4A00023E4DE9
:083D4D00302906740A251EF559
:013D55001E4F
:0A3D5600E51E6006E51E24F350038D
:033D6000753C00AF
:063D6300300F0AE53EB539
:043D69001E028003B3
:033D6D00753C00A2
:043D7000851E3E026C
:023D74003E4DC2
:073D7600E4A22933F51E024F
:023D7D003E4DB9
:063D7F00302904051E05B9
:013D85001E1F
:033D8600023E4DAD
:083D8900302906E51E2404F5B3
:013D91001E13
:033D9200023E4DA1
:083D95003029067408251EF513
:013D9D001E07
:033D9E00023E4D95
:083DA100302906740A251EF505
:013DA9001EFB
:033DAA00023E4D89
:083DAD003029067414251EF5EF
:013DB5001EEF
:033DB600023E4D7D
:083DB9003029067428251EF5CF
:013DC1001EE3
:033DC200023E4D71
:083DC5003029067450251EF59B
:013DCD001ED7
:093DCE00E51E249C5003753C0025
:063DD700300F0AE53FB5C4
:043DDD001E0280033F
:033DE100753C002E
:053DE400851E3F806414
:053DE900301F09805F9E
:073DEE00753C00C20F805874
:073DF500300F5375185A74DA
:0A3DFC0033C0E07400C0E07440C062
:0E3E0600E090003A75F04075D00012724575DC
:0C3E1400D00815811581158175353A74B0
:0A3E200036C0E07400C0E07440C03A
:0E3E2A00E090003D75F04075D0001272E27518
:0B3E3800D008158115811581A2209291
:053E430003D20EE4F5BE
:033E480040F54101
:023E4B00B20FB4
:0C3E4D00D0D0D025D001D000D007D00686
:0E3E5900D005D004D003D002D083D082D0F0A8
:033E6700D0E03276
:0E3E6A00C0E0C082C083C0D075D010C2AF755A
:0D3E78008DFE740C258B2402F58BD2AFE576
:063E85002F453060091515
:073E8B002F74FFB52F021593
:013E920030FF
:093E9300E51F24FA5003023F1A56
:053E9C00E51F251F25B4
:053EA1001F903EA67316
:073EA600023EB8023EC60215
:063EAD003ED8023EEA02CD
:053EB3003EFC023F0E81
:063EB80030B003751F0489
:083EBE0030B159751F02805458
:063EC60030B003751F057A
:093ECC0020B14B751F000539D22D
:033ED5000A80421E
:093ED80030B007751F051539D241
:013EE1000AD6
:083EE20020B135751F0080308E
:093EEA0020B007751F001539D244
:013EF3000AC4
:083EF40030B123751F05801E8B
:063EFC0020B003751F0059
:093F020030B115751F050539D217
:033F0B000A800C1D
:063F0E0020B003751F0145
:063F140020B103751F033C
:093F1A00D0D0D083D082D0E03277
:0D3F2300AA82AB83ACF0C002C003C0041240
:0E3F30006090D004D003D002907B1D75F0800D
:0E3F3E00C002C003C0041260B5D004D003D08E
:0C3F4C0002E54424F65012758220C002E9
:0D3F5800C003C00412609BD004D003D0024F
:0A3F6500AD45854482C002C003C0D0
:0E3F6F000474FFC0E0C0051263E415811581E3
:0E3F7D00D004D003D002758220C002C003C061
:0E3F8B000412609BD004D003D0028A828B8384
:0E3F99008CF0C002C003C0041264E6D004D055
:0E3FA70003D002E4BA0007BB0004BC00010412
:0A3FB500FA6022754301754600C052
:0E3FBF00027401C0E0758209122DC9AB821593
:0D3FCD0081D002EB7007C002121AC0D002B2
:033FDA008A8222B6
:0A3FDD00C05985815905810581AAAC
:0C3FE70082AB83ACF0AD590D7E007F4032
:0E3FF300C002C003C004C005C006C00775822E
:0E4001000C122D5FAD82158115811581D00442
:0C400F00D003D002ED7005A859087663BC
:0C401B00E5592402FD7E007F40C002C079
:0D40270003C004C005C006C00775820D125D
:0E4034002D5FAD82158115811581D004D0035A
:0B404200D002ED7006A8590808766354
:0A404D00A85908E624E84009A85924
:074057000808E624C4500B29
:0A405E00A859087663A859080876EF
:0140680063F4
:0E406900C002C003C004126090D004D003D087
:0E40770002907B2075F080C002C003C00412CE
:0C40850060B5D004D003D002A85908E6B2
:0E40910024F65012758220C002C003C0041233
:08409F00609BD004D003D002A5
:0A40A700A85908088605A8590886E4
:0E40B10006C002C003C00474FFC0E0C0058E4C
:0E40BF00821263E415811581D004D003D00273
:0E40CD00758220C002C003C00412609BD004A4
:0E40DB00D003D0028A828B838CF0C002C00317
:0E40E900C0041264E6D004D003D002E4BA0092
:0840F70007BB0004BC0001043A
:0640FF00FA70030241AB60
:06410500A85908B61800DD
:05410B0040030241AB7E
:07411000A8590808B63C00A5
:0541170040030241AB72
:09411C00754300754600C002C0A5
:0C4125004475820C122DC9AB821581D0AC
:0C41310002EB6042C002C04575820D1216
:0E413D002DC9AB821581D002EB602FC002A805
:0C414B005908E6C0E075820A122DC9ABCD
:0C415700821581D002EB6018C002A8594C
:0E4163000808E6C0E075820B122DC9AB82156C
:0641710081D002EB700793
:07417700C002121AC0D002C1
:06417E00A859088644A8C0
:064184005908088645758C
:0A418A004301754600C0027401C035
:0E419400E0758209122DC9AB821581D002EBB5
:0941A2007007C002121AC0D0021D
:0A41AB00A85908E624E84009A859C5
:0741B5000808E624C45005D0
:0541BC00758200800285
:0241C1008A82F0
:0641C300855981D059224C
:0A41C900C059E581F5592404F58181
:0C41D300AA82AB83ACF0AD590D7E007FDA
:0E41DF0040C002C003C004C005C006C0077582
:0E41ED00820E122D5FAD82158115811581D0D5
:0C41FB0004D003D002ED7005A85908762E
:014207006353
:0C420800E5592402FD7E007F40C002C08A
:0D42140003C004C005C006C00775820F126C
:0E4221002D5FAD82158115811581D004D0036B
:0B422F00D002ED7006A8590808766365
:0A423A00A85908E624E84009A85935
:074244000808E624C4500B3A
:0A424B00A859087663A85908087600
:014255006305
:0E425600C002C003C004126090D004D003D098
:0E42640002907B2375F080C002C003C00412DC
:0C42720060B5D004D003D002A85908E6C3
:0E427E0024F65012758220C002C003C0041244
:08428C00609BD004D003D002B6
:0A429400A85908088605A8590886F5
:0E429E0006C002C003C00474FFC0E0C0058E5D
:0E42AC00821263E415811581D004D003D00284
:0E42BA00758220C002C003C00412609BD004B5
:0E42C800D003D0028A828B838CF0C002C00328
:0E42D600C0041264E6D004D003D002E4BA00A3
:0842E40007BB0004BC0001044B
:0642EC00FA700302441504
:0642F200A85908B61800EF
:0542F800400302441523
:0742FD00A8590808B63C00B7
:05430400400302441516
:0A430900754300E5592403FB7C0016
:0E4313007D40C002C003C004C00575820C12BC
:0E4321002D5FAB82158115811581D002EB70E6
:04432F00030243E161
:0C433300E5592404FB7C007D40C002C062
:0E433F0003C004C00575820D122D5FAB821500
:0D434D008115811581D002EB70030243E160
:0C435A00C002A859080808E6C0E07582FF
:0E4366000E122DC9AB821581D002EB606EC025
:0C43740002E5592404F8E6C0E075820F51
:0E438000122DC9AB821581D002EB6055C00230
:0C438E00C04475820C122DC9AB82158151
:0C439A00D002EB6042C002C04575820DED
:0E43A600122DC9AB821581D002EB602FC00230
:0C43B400A85908E6C0E075820A122DC965
:0C43C000AB821581D002EB6018C002A88F
:0C43CC00590808E6C0E075820B122DC9EC
:0943D800AB821581D002EB7007E5
:0743E100C002121AC0D00255
:0643E800A859088644A854
:0643EE0059080886457520
:0A43F4004301754600C0027401C0C9
:0E43FE00E0758209122DC9AB821581D002EB49
:09440C007007C002121AC0D002B0
:0A441500A85908E624E84009A85958
:07441F000808E624C4500563
:05442600758200800218
:02442B008A8283
:06442D00855981D05922DF
:0A443300C059E581F5592406F58112
:0D443D00AA82AB83ACF0C002C003C0041221
:0E444A006090D004D003D002907B2675F080E5
:0E445800C002C003C0041260B5D004D003D06F
:0E446600028A828B838CF0C002C003C0041255
:0E44740064E6D004D003D002E4BA0007BB0017
:0544820004BC00010470
:06448700FA700302472E4B
:0A448D00C0027445C0E07400C0E0F6
:0E4497007440C0E090004475F0401233D7AB83
:0E44A50082158115811581D002EB7005F5821C
:0344B3000247308D
:0C44B600A8590888037C007D40C002C0AB
:0E44C20000C003C004C00575820A122D5FAB56
:0E44D00082158115811581D000D002EB70039A
:0344DE000245BBD9
:0C44E100E5592404FB8B047D007E40C0E4
:0E44ED0002C003C000C004C005C00675820BEB
:0E44FB00122D5FAC82158115811581D000D085
:0945090003D002EC70030245BB73
:0E451200740128FC7D007E40C002C003C00082
:0E452000C004C005C00675820C122D5FAC826F
:0E452E00158115811581D000D003D002EC70EC
:04453C00030245BB76
:0E45400074012BFC7D007E40C002C003C00051
:0E454E00C004C005C00675820D122D5FAC8240
:0E455C00158115811581D000D003D002EC60CE
:0E456A0050740228FC7D007E40C002C003C0D9
:0E45780000C004C005C00675820E122D5FAC97
:0E45860082158115811581D000D003D002EC82
:0E45940060250B0B7C007D40C002C000C00300
:0E45A200C004C00575820F122D5FAB8215811B
:0B45B00015811581D000D002EB700BCC
:0B45BB00C002C000121AC0D000D002E5
:0A45C6008603E544B5030EE5592411
:0B45D00004F98704E545B5040280698A
:0C45DB00740128F98704E544B50422E5CA
:0C45E700592404FD74012DFEC000A8063C
:0C45F3008607D000E545B5070CA703A91A
:0945FF00058705A906A705803314
:0D460800740228FDC000A805A604D000E53E
:0C461500592404FC74022CFD74012CFEDE
:0E462100C000A8068607D000C000A805A607A6
:0C462F00D000A703A9048703A906A70375
:08463B00A644E5592404F9A787
:014643004531
:0E4644008603C002C000C00375820A122DC991
:0E465200AB821581D000D002EB700302470549
:0C466000E5592404F98703C002C000C023
:0E466C0001C00375820B122DC9AB821581D0DF
:0B467A0001D000D002EB7003024705E6
:0E468500740128FBC000A8038603D000C00209
:0E469300C000C001C00375820C122DC9AB829D
:0E46A1001581D001D000D002EB6059740129C0
:0E46AF00FBC000A8038603D000C002C000C0FC
:0E46BD0001C00375820D122DC9AB821581D08C
:0E46CB0001D000D002EB603208088603C00266
:0E46D900C001C00375820E122DC9AB8215817F
:0E46E700D001D002EB601709098703C002C0A2
:0E46F5000375820F122DC9AB821581D002EB26
:0247030070073D
:07470500C002121AC0D0022D
:0A470C00754301754600C0027401F8
:0E471600C0E0758209122DC9AB821581D00258
:0A472400EB7007C002121AC0D002A9
:02472E008A827D
:06473000855981D05922D9
:0D473600AA82AB83ACF0C002C003C0041225
:0E4743006090D004D003D002907B2F75F080E0
:0E475100C002C003C0041260B5D004D003D073
:0E475F00028A828B838CF0C002C003C0041259
:0E476D0064E6D004D003D002E4BA0007BB001B
:05477B0004BC00010474
:0C478000FA601E754300C002E4C0E07542
:0E478C008209122DC9AB821581D002EB700795
:07479A00C002121AC0D00298
:0347A1008A8222E7
:0D47A400AA82AB83ACF0C002C003C00412B7
:0E47B1006090D004D003D002907B3875F08069
:0E47BF00C002C003C0041260B5D004D003D005
:0E47CD00028A828B838CF0C002C003C00412EB
:0E47DB0064E6D004D003D002E4BA0007BB00AD
:0547E90004BC00010406
:0C47EE00FA6054C3E54664809498504B78
:0A47FA0074182546F546B41823E5AF
:074804004624F5F546C3E56B
:09480B00449533500D7418C39557
:0448140033254425DF
:0548180046F546800991
:06481D00E544C3953325BC
:0348230046F54611
:0C482600754304C0027404C0E0758209F0
:0E483200122DC9AB821581D002EB7007C002B7
:05484000121AC0D002B5
:034845008A822242
:0E484800AA82AB83ACF0E4BA0007BB0004BC4C
:034856000001045A
:06485900FD700302496E30
:0A485F00E5426007E542B4017080F5
:014869003717
:0C486A00754201907B4175F080C002C0D7
:0E48760003C004C0051216D2D005D004D00332
:0C488400D002754300758200C002C00322
:0E489000C004C005121A76D005D004D003D0A3
:03489E0002805342
:0C48A100754202907B4A75F080C002C096
:0E48AD0003C004C0051216D2D005D004D003FB
:0C48BB00D002754300758200C002C003EB
:0E48C700C004C005121A76D005D004D003D06C
:0348D50002801C42
:0C48D800754200907B5375F080C002C058
:0E48E40003C004C0051216D2D005D004D003C4
:0248F200D002F2
:0E48F4009001F4C002C003C004C0051218BF3A
:0E490200D005D004D003D002C002C003C00410
:0C491000C005C042758200122DC9AE82A5
:0E491C001581D005D004D003D002EE7013C078
:0E492A0002C003C004C005121AC0D005D0049C
:04493800D003D002D6
:0C493C00C002C003C004C005C043758267
:0E49480009122DC9AE821581D005D004D0030E
:0E495600D002EE7013C002C003C004C00512F0
:0A4964001AC0D005D004D003D00221
:0E496E00C002C003C004C005126090D005D086
:0A497C0004D003D002E5426007E515
:0649860042B40138801B61
:0E498C00907B5C75F080C002C003C004C005C3
:0D499A001260B5D005D004D003D0028034E7
:0E49A700907B6575F080C002C003C004C0059F
:0D49B5001260B5D005D004D003D0028019E7
:0E49C200907B6E75F080C002C003C004C0057B
:0B49D0001260B5D005D004D003D00267
:0E49DB008A828B838CF0C0051264E6D0058DB5
:0249E900822228
:0E49EB00AA82AB83ACF0E4BA0007BB0004BCA8
:0349F900000104B6
:0C49FC00FD6038B210C002C003C004C04F
:0B4A080005E4A21033C0E0758201122B
:0E4A13002DC9AE821581D005D004D003D0028B
:0E4A2100EE7013C002C003C004C005121AC01C
:084A2F00D005D004D003D00231
:0E4A3700C002C003C004C005126090D005D0BC
:0C4A450004D003D00230101B907B77756A
:0E4A5100F080C002C003C004C0051260B5D0E2
:094A5F0005D004D003D002801937
:0E4A6800907B8075F080C002C003C004C005C2
:0B4A76001260B5D005D004D003D002C0
:0E4A81008A828B838CF0C0051264E6D0058D0E
:024A8F00822281
:0E4A9100AA82AB83ACF0E4BA0007BB0004BC01
:034A9F000001040F
:0C4AA200FD6038B214C002C003C004C0A4
:0B4AAE0005E4A21433C0E0758206127C
:0E4AB9002DC9AE821581D005D004D003D002E5
:0E4AC700EE7013C002C003C004C005121AC076
:084AD500D005D004D003D0028B
:0E4ADD00C002C003C004C005126090D005D016
:0C4AEB0004D003D00230141B907B8975AE
:0E4AF700F080C002C003C004C0051260B5D03C
:094B050005D004D003D002801990
:0E4B0E00907B9275F080C002C003C004C00509
:0B4B1C001260B5D005D004D003D00219
:0E4B27008A828B838CF0C0051264E6D0058D67
:024B35008222DA
:0E4B3700AA82AB83ACF0E4BA0007BB0004BC5A
:034B450000010468
:0C4B4800FD6038B211C002C003C004C000
:0B4B540005E4A21133C0E075820212DC
:0E4B5F002DC9AE821581D005D004D003D0023E
:0E4B6D00EE7013C002C003C004C005121AC0CF
:084B7B00D005D004D003D002E4
:0E4B8300C002C003C004C005126090D005D06F
:0C4B910004D003D00230111B907B9B75F8
:0E4B9D00F080C002C003C004C0051260B5D095
:094BAB0005D004D003D0028019EA
:0E4BB400907BA475F080C002C003C004C00551
:0B4BC2001260B5D005D004D003D00273
:0E4BCD008A828B838CF0C0051264E6D0058DC1
:024BDB00822234
:0E4BDD00AA82AB83ACF0E4BA0007BB0004BCB4
:034BEB00000104C2
:0C4BEE00FD6051B212C002C003C004C040
:0B4BFA0005E4A21233C0E07582031234
:0E4C05002DC9AE821581D005D004D003D00297
:0E4C1300EE7013C002C003C004C005121AC028
:084C2100D005D004D003D0023D
:0C4C2900201216758200C002C003C004F7
:0D4C3500C005121AABD005D004D003D00288
:0E4C4200C002C003C004C005126090D005D0AF
:0C4C500004D003D00230121B907BAD7525
:0E4C5C00F080C002C003C004C0051260B5D0D5
:094C6A0005D004D003D00280192A
:0E4C7300907BB675F080C002C003C004C0057F
:0B4C81001260B5D005D004D003D002B3
:0E4C8C008A828B838CF0C0051264E6D0058D01
:024C9A00822274
:0A4C9C00C0598581590581AA82AB39
:0A4CA60083ACF0C228AD590D7E006A
:0C4CB0007F40C002C003C004C025C00546
:0E4CBC00C006C007758204122D5FAD821581FF
:0C4CCA0015811581D025D004D003D00244
:0B4CD600ED6008A85908E6249C50057A
:054CE100A8590876143B
:0A4CE600A85908E6249C5005A859BF
:034CF000087663E0
:064CF300A85908B60100FB
:074CF9005005A859087601DF
:0B4D0000E4BA0007BB0004BC00010483
:064D0B00FD7003024EC81A
:0E4D1100C002C003C004C005121B1DD005D097
:054D1F0004D003D002E6
:0E4D2400C00575821EC002C003C004C0051287
:0E4D32001A51D005D004D003D002C002C00335
:0E4D4000C004C005126090D005D004D003D08E
:0E4D4E0002907BBF75F080C002C003C004C09D
:0D4D5C00051260B5D005D004D003D002A828
:0A4D69005908A859088682C002C04C
:0E4D730003C004C0051262B3D005D004D00303
:0E4D8100D002907BC375F080C002C003C00456
:0E4D8F00C0051260B5D005D004D003D002C01C
:0E4D9D0002C003C0041264DFAE82AF83ADF02B
:0E4DAB00D004D003D0028E828F838DF0C00220
:0E4DB900C003C004C0051216D2D005D004D02D
:054DC70003D002D0053D
:0C4DCC00200867C002C003C004C005122C
:0E4DD8001A5AE582D005D004D003D0027050E4
:0A4DE600C296D296E53930E7117548
:0A4DF0003900A85908E624FE503CE3
:064DFA00A85908168036DE
:0C4E0000C374808539F063F08095F05099
:0A4E0C0011753900A85908B66300BB
:084E1600501EA859080680187F
:0E4E1E00758202C002C003C004C005122084C9
:0A4E2C00D005D004D003D002809618
:0E4E3600C002C003C004C005121A5AAE82D0DA
:0C4E440005D004D003D002EE24FF922819
:074E500020080620280302E0
:024E57004D24E8
:0B4E5900C002C003C004C005C0251249
:0C4E64001B1DD025D005D004D003D002C7
:0C4E700075820AC002C003C004C005C067
:054E7C00251219C2D04F
:0C4E810025D005D004D003D002C002C030
:0A4E8D0003C004C005C025A85908A1
:0E4E9700E6C0E0758204122DC9AE821581D0EE
:0C4EA50025D005D004D003D002EE701719
:0B4EB100C002C003C004C005C02512F1
:0C4EBC001AC0D025D005D004D003D002CD
:0B4EC800C002C003C004C005C02512DA
:0C4ED3006090D025D005D004D003D002A0
:0E4EDF00907BC775F080C002C003C004C00500
:064EED00C0251260B5D0E3
:0A4EF30025D005D004D003D002A89A
:0A4EFD005908A859088682C002C0B7
:0B4F070003C004C005C0251262B3D037
:0C4F120025D005D004D003D00275826DBC
:0B4F1E00C002C003C004C005C0251283
:0C4F2900609BD025D005D004D003D0023E
:0B4F35008A828B838CF0C005C025121F
:074F400064E6D025D0053026
:074F470028057582008002BD
:024F4E008D8252
:064F5000855981D05922B1
:0E4F5600AA82AB83ACF0E4BA0007BB0004BC37
:034F640000010445
:064F6700FD7003024FF291
:064F6D00B21330131B908B
:0E4F73007BCD75F080C002C003C004C00512E3
:0C4F810016D2D005D004D003D002801955
:0E4F8D00907BD675F080C002C003C004C00542
:0B4F9B001216D2D005D004D003D002C3
:0E4FA6009001F4C002C003C004C0051218BF81
:0E4FB400D005D004D003D002C002C003C00458
:0C4FC200C005E4A21333C0E075820512A4
:0E4FCE002DC9AE821581D005D004D003D002CB
:0E4FDC00EE7013C002C003C004C005121AC05C
:084FEA00D005D004D003D00271
:0E4FF200C002C003C004C005126090D005D0FC
:0C50000004D003D00230131B907BDF753E
:0E500C00F080C002C003C004C0051260B5D021
:09501A0005D004D003D002801976
:0E502300907BE875F080C002C003C004C00599
:0B5031001260B5D005D004D003D002FF
:0E503C008A828B838CF0C0051264E6D0058D4D
:02504A008222C0
:0E504C00AA82AB83ACF0E4BA0007BB0004BC40
:03505A000001044E
:0C505D00FD6038B216C002C003C004C0E1
:0B50690005E4A21633C0E075821012AF
:0E5074002DC9AE821581D005D004D003D00224
:0E508200EE7013C002C003C004C005121AC0B5
:08509000D005D004D003D002CA
:0E509800C002C003C004C005126090D005D055
:0C50A60004D003D00230161B907BF17583
:0E50B200F080C002C003C004C0051260B5D07B
:0950C00005D004D003D0028019D0
:0E50C900907BFA75F080C002C003C004C005E1
:0B50D7001260B5D005D004D003D00259
:0E50E2008A828B838CF0C0051264E6D0058DA7
:0250F00082221A
:0E50F200AA82AB83ACF0E4BA0007BB0004BC9A
:03510000000104A7
:0C510300FD6038B217C002C003C004C039
:0B510F0005E4A21733C0E07582111206
:0E511A002DC9AE821581D005D004D003D0027D
:0E512800EE7013C002C003C004C005121AC00E
:08513600D005D004D003D00223
:0E513E00C002C003C004C005126090D005D0AE
:0C514C0004D003D00230171B907C0375C8
:0E515800F080C002C003C004C0051260B5D0D4
:0951660005D004D003D002801929
:0E516F00907C0C75F080C002C003C004C00527
:0B517D001260B5D005D004D003D002B2
:0E5188008A828B838CF0C0051264E6D0058D00
:02519600822273
:0E519800AA82AB83ACF0BA0008BB0005BC00D5
:0351A60002800381
:0351A9000253515D
:0C51AC00C20875821EC002C003C00412BD
:0851B8001A51D004D003D0020B
:0E51C000C002C003C004126090D004D003D01F
:0E51CE0002907C1575F080C002C003C0041270
:0C51DC0060B5D004D003D002C3E54094BD
:0C51E800A0E54194055069C002C003C05E
:0C51F40004743CC0E0E4C0E0854082850B
:0C5200004183127422AD82AE831581152B
:0E520C0081D004D003D002C002C003C004C091
:0C521A0005743CC0E0E4C0E085408285E3
:0C522600418312737FAE82AF83158115A7
:0E52320081D005D004D003D0028E82C002C00D
:0E52400003C00474FFC0E0C0051263E41581D2
:0A524E001581D004D003D002806D5A
:0A525800C3E5409460E5419427503F
:0E5262004DC002C003C00474A0C0E07405C0BB
:08527000E085408285418312B4
:0E527800737FAD82AE8315811581D004D00303
:0E528600D0028D82C002C003C004126100D0AD
:0E52940004D003D002907C1975F080C002C0D7
:0E52A20003C0041260B5D004D003D002801502
:0D52B000907C1E75F080C002C003C0041287
:0852BD0060B5D004D003D0025B
:0E52C500C002C003C0041264DFAD82AE83AF2E
:0E52D300F0D004D003D0028D828E838FF0C005
:0E52E10002C003C0041216D2D004D003D002C3
:0E52EF00758201C002C003C0041220DED0048C
:0E52FD00D003D002900005C002C003C004120E
:0D530B0018BFD004D003D002C296D2962065
:0C5318000816C002C003C004121A5AE5B7
:0C53240082D004D003D00270030251C0FC
:0E533000C002C003C004121B1DD004D003D065
:0E533E000275820AC002C003C0041219C2D058
:05534C0004D003D002B3
:0E535100C002C003C004126090D004D003D08C
:0E535F0002907C2475F080C002C003C00412CE
:0E536D0060B5D004D003D0028A828B838CF00E
:07537B001264E675820022B6
:0E538200AA82AB83ACF0BA0056BB0053BC004D
:0553900050D2287D0051
:0B539500ED907C2D93FEBEFF028024F3
:0C53A00074012D907C2D93FFC005C025EA
:0C53AC00C0078E82122DC9AE821581D080
:0853B80025D005EE7002C228A9
:0453C0000D0D80D17E
:0953C400758214C025121923D0D2
:0553CD002530280B90C3
:0A53D2007C5275F0801216D28003A1
:0353DC00121AC0E2
:0253DF0080FE4E
:0E53E100C002C003C004126090D004D003D0FC
:0E53EF0002907C5B75F080C002C003C0041207
:0E53FD0060B5D004D003D0028A828B838CF07E
:07540B001264E67582002225
:0E541200AA82AB83ACF0BA000BBB0008BC0052
:0454200005122D1E26
:0254240080FE08
:0E542600C002C003C004126090D004D003D0B6
:0E54340002907C6475F080C002C003C00412B8
:0E54420060B5D004D003D0028A828B838CF038
:075450001264E675820022E0
:0D545700AA82AB83ACF0C002C003C00412F7
:0E5464006090D004D003D002907C6D75F08073
:0E547200C002C003C0041260B5D004D003D045
:0E548000028A828B838CF01264E67582002211
:0A548E00C059E581F5592411F5819C
:0A549800E54424E84006E54524C47D
:0254A2005006B2
:0654A40075440875450087
:0B54AA00E559240FF8760075821E12F1
:0E54B5001A5175820A1219C274E6C0E0740121
:0E54C300C0E0907C8575F08012171C158115D5
:0E54D1008174E6C0E07401C0E0907C8E75F03E
:0E54DF008012171C158115819001F41218BF60
:0954ED00A859087600121B1D905D
:0C54F6007C76E493FC740193FDE55924DE
:0E55020002FE8E077B007A40C004C005C00682
:0A5510007423C0E07455C0E0C0042D
:09551A00C0058F828B838AF02208
:0E552300D006D005D0048E027B007C40C0066E
:0E55310074FAC0E07401C0E08A828B838CF0B3
:0E553F0012171C15811581D006C006E4C0E0CD
:0D554D0075821312155F1581D0068E02E5E0
:0A555A00592411F8A606E5592410A3
:05556400F8A6068E050B
:065569003008030257AEFA
:0E556F00C002C005121A5AE582D005D00260B3
:04557D00030257AE20
:0E558100C296D296C002C005121B27D005D0DC
:0E558F0002758200C002C0051220B1D005D006
:09559D0002E559240BF8A639E5DA
:0C55A60059240BF8C3748086F063F08079
:0755B20095F040030256C111
:0C55B900C005753900907C84E493FF8FDE
:0A55C500053395E0FE1DBDFF011E39
:0C55CF00A859088604E63395E0FBC3EC05
:0E55DB009DEB64808EF063F08095F0D005406B
:0455E900030256B3B0
:0A55ED00A85908E559240BF9E72638
:0C55F700F6A85908C3E664808FF063F04A
:0B5603008095F04006A85908EF14F64F
:0E560E00C005758204C002C005121950D005F7
:0D561C00D002C002C005E4C0E075820E128D
:0C562900155F1581D005D002A85908C2F9
:0C563500D575F002E630E704B2D5F404AD
:0E564100A430D50AF42401C5F0F43400C5F0FD
:0A564F002476F582747C35F0F583B3
:0E565900E493FB740193FC8A067F007D40C041
:0C56670002C003C004C0057481C0E074E0
:0C56730056C0E0C003C0048E828F838DFF
:02567F00F02217
:0C568100D005D004D003D002E55924115C
:0E568D00F886037C007D40C002C00574FAC0A0
:0E569B00E07401C0E08B828C838DF012171C2E
:0A56A90015811581D005D002D0054F
:0E56B30075821EC002C005121A51D005D00229
:0C56C100E559240BF8E620E703025569C8
:0A56CD00753900A85908C3748086DF
:0B56D700F063F08095F0400302579D47
:0A56E200A85908E559240BF9E72642
:0A56EC00F6A85908E630E705A859B2
:0356F60008760033
:0E56F900C002758204C002C005121950D0050F
:0D570700D002C002C005E4C0E075820F12A0
:0C571400155F1581D005D002A85908C20D
:0C572000D575F002E630E704B2D5F404C1
:0E572C00A430D50AF42401C5F0F43400C5F011
:0A573A002476F582747C35F0F583C7
:0C574400E493FB740193FCE5592410F879
:0E57500086067F007A40C002C003C004C00578
:0A575E007471C0E07457C0E0C0038E
:09576800C0048E828F838AF022B6
:0E577100D005D004D003D0028D027B007C4016
:0E577F00C002C00574FAC0E0E4C0E08A828B6C
:0E578D00838CF012171C15811581D005D002F7
:02579B00D0023A
:0E579D0075821EC002C005121A51D005D0023E
:0357AB000255693B
:0A57AE00C296D29610080302589923
:0D57B80075820A1219C2E4C0E07582111258
:0C57C500155F1581A85908C2D575F002C7
:0857D100E630E704B2D5F40450
:0E57D900A430D50AF42401C5F0F43400C5F064
:0A57E7002476F582747C35F0F5831A
:0C57F100E493FA740193FBC003740DC034
:0C57FD00E07458C0E0C002C0039000003F
:0458090075F0002214
:0C580D00AA82D003E559240FF8A6027A05
:01581900008E
:0E581A00BA0335907C84E493FB3395E0FC1BCD
:04582800BBFF011CA5
:0C582C00A859088605E63395E0FEC3EDA0
:0E5838009BEE64808CF063F08095F0500D9034
:0C5846007C9675F080C0021216D2D002D1
:0E585200C002E4C0E075822012155F1581D0FF
:0E58600002900050C0021218BFD002C002E435
:0D586E00C0E075821112155F1581D0029007
:0E587B000050C0021218BFD0020AC296D29688
:03588900BA06005C
:05588C00500302581A50
:0658910030070302581A63
:02589700800F80
:0D589900907C9F75F0801216D2758214125B
:0258A6001923C4
:0C58A800121B1DE559240FF8E6700302E6
:0258B4005BC3D4
:0758B600E543B40102800389
:0358BD000259CCC1
:0E58C0009001901218BF74B4C0E07401C0E0F3
:0E58CE00907CA875F08012171C158115819032
:0958DC0001901218BFC3E54495C8
:0C58E50033503874B4C0E07401C0E0908F
:0D58F1007CB175F08012171C158115819097
:0E58FE0001901218BF74B4C0E07401C0E090B5
:0D590C007CBA75F08012171C158115819072
:0759190001901218BF801B72
:0E59200074B4C0E07401C0E0907CC375F080E8
:0D592E0012171C158115819001901218BFF1
:0A593B00126090907CCC75F0801291
:0C59450060B5E54424F65006758220127F
:02595100609B59
:0A595300AA4585448274FFC0E0C03D
:0E595D00021263E41581158175822012609B91
:0E596B001264DFAA82AB83ACF074B4C0E074A7
:0E59790001C0E08A828B838CF012171C15810E
:0E5987001581C296D2969001F41218BF7A00D4
:03599500BA040051
:055998004003025BC3A7
:0E599D00C296D296758200C002121A76D0020F
:0E59AB00900096C0021218BFD002758201C093
:0E59B90002121A76D002900096C0021218BF99
:0559C700D0020A80C9B6
:0759CC00E543B4040280036F
:0359D300025B7202
:0E59D6009001901218BF758200121A7674B4F8
:0D59E400C0E07401C0E0907CCF75F080122F
:0859F100171C158115817A00D5
:0359F900BA0400ED
:0E59FC00502FC296D296758201C002121A7602
:0E5A0A00D002900096C0021218BFD002758222
:0E5A180000C002121A76D002900096C0021250
:075A260018BFD0020A80CC7A
:0A5A2D00AA33E559240CFB7C007D30
:0E5A370040C002C003C004C00590003675F0E8
:0E5A4500401272E2158115811581D0027B009E
:0C5A5300E546FC3395E0FD740B2CFCE4F0
:0E5A5F003DFD8B067F00C3EE9CEF64808DF052
:0E5A6D0063F08095F050230ABA181C7A00E509
:0C5A7B0059240CFC7D007E408C828D8341
:0D5A87008EF0C002C00312692ED003D002C1
:035A94000B80BCC8
:0D5A9700907CD875F08012275A9001F4120F
:065AA40018BF126090E53E
:0C5AAA0059240CFA7B007C408A828B831C
:0D5AB6008CF01265A9E582FA24F850030275
:025AC3005B3155
:075AC500EA2A2A905ACC7373
:075ACC00025B31025AE40203
:065AD3005AEF025AFA022C
:065AD9005B05025B1002F8
:055ADF005B1B025B26C9
:0B5AE400907CF375F0801260B5804BE1
:0B5AEF00907CF775F0801260B58040DD
:0B5AFA00907CFB75F0801260B58035D9
:0B5B0500907CFF75F0801260B5802AD4
:0B5B1000907D0375F0801260B5801FCF
:0B5B1B00907D0775F0801260B58014CB
:0B5B2600907D0B75F0801260B58009C7
:095B3100907D0F75F0801260B543
:0A5B3A00AA4585448274FFC0E0C054
:0E5B4400021263E4158115811264DFAA82ABA0
:0E5B520083ACF074C8C0E07401C0E08A828B9E
:0E5B6000838CF012171C158115819007D0124E
:045B6E0018BF80518B
:0E5B72009001901218BF74B4C0E07401C0E03E
:0E5B8000907D1375F08012171C158115817A27
:015B8E000016
:035B8F00BA040055
:0E5B9200502FC296D296758201C002121A766A
:0E5BA000D002900096C0021218BFD00275828B
:0E5BAE0000C002121A76D002900096C00212B9
:075BBC0018BFD0020A80CCE3
:0E5BC3009000961218BF74DCC0E07401C0E0C0
:0E5BD100907D1C75F08012171C1581158185C2
:055BDF005981D059229C
:0A5BE400C059E581F5592413F5813D
:0E5BEE0075821E121A5175820A1219C274E6CF
:0D5BFC00C0E07401C0E0907C8575F080125F
:0E5C0900171C1581158174E6C0E07401C0E01F
:0E5C1700907D4075F08012171C15811581904C
:0C5C250001F41218BFA8590808760012FC
:0D5C31001B1D907D25E493FB740193FCE5A1
:0C5C3E00592403FD8D067F007A40C0034E
:0A5C4A00C004C0057461C0E0745C82
:0D5C5400C0E0C003C0048E828F838AF0225E
:0E5C6100D005D004D0038D027B007C40C0052E
:0E5C6F0074FAC0E07401C0E08A828B838CF06E
:0C5C7D0012171C15811581D0058D02E561
:0A5C8900592410F8A605E559240F70
:0B5C9300F8A605E559240EF8A605E56B
:0A5C9E00592411F8A605E559240D5C
:035CA800F8A60556
:0E5CAB00C002E4C0E075821312155F1581D0AF
:015CB90002E8
:065CBA00300803025ECE7B
:0E5CC000C002121A5AE582D0026003025ECEC4
:0E5CCE00C296D296C002121B27D00275820029
:0C5CDC00C0021220B1D002E559240CF8DF
:0A5CE800A639E559240CF8C37480B6
:0C5CF20086F063F08095F04003025DEF47
:0C5CFE00753900907D3FE493FB8B073369
:085D0A0095E0FD1FBFFF011D24
:0C5D1200A85908088606E63395E0FCC39B
:0E5D1E00EE9FEC64808DF063F08095F0400302
:035D2C00025DE530
:0A5D2F00A8590808E559240CF9E70B
:0C5D390026F6A8590808C3E664808BF029
:0C5D450063F08095F04007A8590808EBB7
:025D510014F646
:0E5D5300758204C002121950D002C002E4C0D2
:0C5D6100E075820E12155F1581D002A8BB
:0C5D6D00590808C2D575F002E630E704C2
:045D7900B2D5F404A7
:0E5D7D00A430D50AF42401C5F0F43400C5F0BA
:0A5D8B002425F582747D35F0F583C0
:0E5D9500E493FC740193FD8A067F007B40C0FE
:0A5DA30002C004C00574BBC0E07428
:0C5DAD005DC0E0C004C0058E828F838BB7
:025DB900F022D6
:0C5DBB00D005D004D002E5592410F88671
:0E5DC700037C007D40C00274FAC0E07401C08D
:0E5DD500E08B828C838DF012171C15811581D6
:025DE300D002EC
:0A5DE50075821EC002121A51D0028E
:0C5DEF00E559240CF8E620E703025CBA3A
:0A5DFB00753900A8590808C3748028
:0C5E050086F063F08095F04003025EC15F
:0A5E1100A8590808E559240CF9E728
:0B5E1B0026F6A8590808E630E706A8A4
:055E2600590808760098
:0E5E2B00758204C002121950D002C002E4C0F9
:0C5E3900E075820F12155F1581D002A8E1
:0C5E4500590808C2D575F002E630E704E9
:045E5100B2D5F404CE
:0E5E5500A430D50AF42401C5F0F43400C5F0E1
:0A5E63002425F582747D35F0F583E7
:0C5E6D00E493FB740193FCE559240FF84A
:0D5E790086057E007F40C002C003C0047497
:0A5E860098C0E0745EC0E0C003C0E5
:085E9000048D828E838FF02245
:0C5E9800D004D003D002E559240EF88697
:0E5EA400067B007C40C00274FAC0E0E4C0E05F
:0E5EB2008E828B838CF012171C15811581D007
:015EC00002DF
:0D5EC10075821EC002121A51D002025CBA96
:0A5ECE00C296D29610080302603D50
:0E5ED80075821EC002121A51D00275820AC0D5
:0E5EE600021219C2D002C002E4C0E07582119F
:0C5EF40012155F1581D002A8590808C2E1
:0C5F0000D575F002E630E704B2D5F404D9
:0E5F0C00A430D50AF42401C5F0F43400C5F029
:0A5F1A00FBACF0EB2425F582EC341B
:0C5F24007DF583E493FD740193FEC00240
:0C5F3000C003C004C005C006744BC0E0F4
:0C5F3C00745FC0E0C005C0069000007556
:035F4800F0002244
:0C5F4B00D006D005D004D003D002A85925
:035F5700087600C9
:0A5F5A00A85908B6036DC002EB243D
:095F640025F582EC347DF583E59E
:0C5F6D00592412F8E493F674019308F62E
:0C5F7900E5592411F886057F007A40C02D
:0A5F850002C003C00474A5C0E0745C
:0A5F8F005FC0E0E5592412F8E6C0F7
:0C5F9900E008E6C0E08D828F838AF022D1
:0C5FA500D004D003D002E559240DF8868A
:0E5FB100057A007E408D828A838EF0C002C089
:0E5FBF0003C0041216D2D004D003D002D002C8
:0D5FCD00C002C003C004E4C0E075822012D1
:0E5FDA00155F1581D004D003D002900050C096
:0E5FE80002C003C0041218BFD004D003D002C0
:0D5FF600C002C003C004E4C0E075821112B7
:0E600300155F1581D004D003D002900050C06C
:0E60110002C003C0041218BFD004D003D00296
:0A601F00A8590806C296D296200880
:0760290024A85908B6060087
:056030005003025F5A5D
:06603500300703025F5A70
:02603B008011D2
:0D603D00907C9F75F0801216D275821412AF
:04604A00192380276F
:0E604E00907D3FE493FB3395E0FC1BBBFF010C
:01605C001C27
:0C605D00A85908088605E63395E0FEED22
:09606900B50306EEB50402800344
:03607200025CAB22
:0E60750074DCC0E07401C0E0907D1C75F0800A
:0B60830012171C15811581855981D072
:02608E00592295
:037B1D00091B0041
:037B2000091C003D
:037B2300091D0039
:097B2600095374656C6C656E0076
:097B2F000920417573202020009B
:097B3800092031D74175732000CA
:097B41001154696D6572162000F3
:097B4A00114E69636874731600A2
:097B5300115765636B65721600A1
:097B5C00094D6F6475730A5700AE
:097B6500094D6F6475730A5400A8
:097B6E00094D6F6475730A2D00C6
:097B770009446174756D0A0D00EA
:097B800009446174756D0A0C00E2
:097B89000946656965720A0D00E8
:097B92000946656965720A0C00E0
:097B9B000954656D700B0A0D0020
:097BA4000954656D700B0A0C0018
:097BAD00094B6E6F70660A0D00B1
:097BB600094B6E6F70660A0C00A9
:047BBF000920090090
:047BC3006D696E007A
:067BC70009574C5A0A00A8
:097BCD0011546F6E1620202000F7
:097BD60011526164696F16200070
:097BDF0009574D540A546F6E0061
:097BE80009574D540A5261640072
:097BF100095745413A200C20001F
:097BFA00095745413A200D200015
:097C0300094654413A200C20000E
:097C0C00094654413A200D200004
:047C15000909090050
:057C19002054672E005D
:067C1E003E3120576F000B
:097C240009444346656D706600D9
:0E7C2D0000000101020103010414050106011B
:0E7C3B000705081E09000A080B000C070D00C3
:097C49000E060F0010011101FFED
:097C5200092E2E2E2E2E4F6B0080
:097C5B00094772756E6473740030
:097C6400095265736574202000CB
:097C6D0009167A7572FC636B00C4
:027C7600233FAA
:027C7800DD3FEE
:027C7A00C941FE
:027C7C0033448F
:027C7E00364787
:027C8000A44717
:027C8200575455
:017C840007F8
:097C8500022D2D2D2D2D2D0300E3
:087C8E00095765636B65720084
:097C960009205765636B6572005B
:097C9F002020D7D7D7D720200000
:097CA80067657374656C6C74006F
:097CB100617566202020202000EE
:097CBA004D6F7267656E3A2000FF
:097CC3006175663A2020202000C2
:037CCC0020110084
:097CCF002031D741757316200025
:0E7CD8004EE46368737465720A5765636B2D22
:0D7CE6002020200A7465726D696E3A20003E
:047CF3004D6F0B00C6
:047CF70044690B00D1
:047CFB004D690B00C4
:047CFF00446F0B00C3
:047D030046720B00B9
:047D070053610B00B9
:047D0B00536F0B00A7
:047D0F003F3F0B00E7
:097D1300202041757316202000A8
:097D1C002020202020202020005E
:027D25004848CC
:027D2700EB4926
:027D2900914A7D
:027D2B00374BD4
:027D2D00DD4B2C
:027D2F009C4C6A
:027D3100564FAB
:027D33004C50B2
:027D3500F2500A
:027D3700985161
:027D3900825373
:027D3B001254E0
:027D3D00575499
:017D3F000D36
:087D40000945696E73742E0001
:0700F200754F007550007509
:0200F9005800AD
:07609000754F007558002256
:046097008558822284
:09609B00AA8274F8255850012274
:0860A400E558244FF8A602059F
:0460AC0058E5582437
:0560B0004FF87600220C
:0E60B500AA82AB83ACF0BA0007BB0004BC00AB
:0260C3000122B8
:0E60C5008A828B838CF01273C9FD60188D8265
:0E60D300C002C003C00412609BD004D003D0F2
:0860E100020ABA00DF0B80DCAB
:0160E9002294
:0A60EA00AA82C3E5589A5002AA5892
:0760F400E558C39AF558249A
:0560FB004FF8760022C1
:0E610000AA8275F064EA84FB74302BFBBB307E
:03610E00028025E7
:0E6111008B82C00212609BD00275F064EA849B
:0E611F00AAF075F00AEA84FC74302CFBF582BD
:09612D00C00212609BD002801F29
:0E61360075F064EA84AAF075F00AEA84FC743D
:08614400302CFBBB3002800986
:09614C008B82C00212609BD0029C
:0E61550075F00AEA84AAF074302AFBF5820283
:02616300609B3F
:0E616500AA82AB838B048C05EDC4540FFE742C
:066173000F5EFDBD0A00F5
:0E617900501674302DF582C002C003C004120F
:0A618700609BD004D003D002801406
:0E61910074372DF582C002C003C00412609B5B
:06619F00D004D003D00281
:0861A5008C0553050FBD0A0033
:0E61AD00501274302DF582C002C00312609BA8
:0661BB00D003D0028010A9
:0E61C10074372DF582C002C00312609BD0031C
:0261CF00D002FC
:0E61D1008A047E008C05EDC4540FFC740F5C34
:0461DF00FDBD0A00F8
:0E61E300501274302DF582C002C00312609B72
:0661F100D003D002801073
:0E61F70074372DF582C002C00312609BD003E6
:02620500D002C5
:0A6207007B008A0553050FBD0A0055
:0A621100500874302DF58202609BE6
:08621B0074372DF58202609B2F
:0E622300E582FA30E72375822DC00212609BDF
:0E623100D002BA801275823112609B758232E3
:09623F0012609B75823802609B1D
:04624800C3E49AFA17
:05624C008A82026100DE
:0E625100E582FA249C500C75822D12609B751C
:05625F00822D02609B8E
:0E62640075F00AEA842430F582C00212609BB5
:0E627200D00275F00AEA84E5F02430F58202CD
:02628000609B21
:0E628200E582FA249C500C75822D12609B75EB
:05629000822D02609B5D
:0E62950075F00AEA842489F582C00212609B2B
:0E62A300D00275F00AEA84E5F02489F5820243
:0262B100609BF0
:0E62B300E582FA249C500C75822D12609B75BA
:0562C100822D02609B2C
:0362C600BA0A0011
:0E62C900500C758220C00212609BD002801023
:0E62D70075F00AEA842430F582C00212609B42
:0262E500D002E5
:0E62E70075F00AEA84E5F02430F58202609B2F
:0E62F500E582FA249C500C75822D12609B7578
:05630300822D02609BE9
:03630800BA0A00CE
:0E630B00500C758220C00212609BD0028010E0
:0E63190075F00AEA842489F582C00212609BA6
:02632700D002A2
:0E63290075F00AEA84E5F02489F58202609B93
:0A633700E582FA24F350030263DB51
:07634100EA2A2A9063487369
:076348000263DB02636F0238
:06634F0063780263810285
:06635500638A026393025B
:06635B00639C0263A50231
:0663610063AE0263B70207
:0663670063C00263C902DD
:02636D0063D2F9
:09636F00907D4875F0800260B5D4
:09637800907D4D75F0800260B5C6
:09638100907D5275F0800260B5B8
:09638A00907D5775F0800260B5AA
:09639300907D5C75F0800260B59C
:09639C00907D6175F0800260B58E
:0963A500907D6675F0800260B580
:0963AE00907D6B75F0800260B572
:0963B700907D7075F0800260B564
:0963C000907D7575F0800260B556
:0963C900907D7A75F0800260B548
:0963D200907D7F75F0800260B53A
:0963DB00907D8475F0800260B52C
:0A63E400C059858159AA82E4BAFF6E
:0263EE000104A8
:0E63F000FB7020C3EA64809498500B8A82C030
:0863FE00031262B3D003800D0D
:0D640600907D8875F080C0031260B5D00352
:0C641300EB7014A859181818B6FF02808E
:01641F000A72
:0A64200075823AC00312609BD0039E
:0A642A00A859181818E4B6FF010481
:0C643400FA7049A859181818C3E66480D3
:0C64400094BC502BEB6014A859181818DD
:0E644C008682C002C0031262B3D003D0028069
:01645A00251C
:0C645B00A8591818188682C002C003124D
:086467006251D003D002801144
:0E646F00907D8875F080C002C0031260B5D029
:03647D0003D00247
:0C648000EA7018E55924FCF8B6FF028011
:01648C000E01
:0E648D0075823AC002C00312609BD003D00299
:0A649B00E55924FCF8B6FF02803436
:0C64A500E55924FCF8C3E6648094BC5068
:0C64B1001EEB600FEA600CE55924FCF8BB
:0764BD0086821262B3801514
:0C64C400E55924FCF88682126251800920
:0964D000907D8875F0801260B522
:0664D900855981D0592213
:0764DF0090004F75F0402210
:0A64E600C059858159C082C083C0EF
:0C64F000F0A85908B6000D08B600090815
:0864FC00B60005758200804521
:026504007D0018
:0B650600ED244FF88606BE0002801F47
:03651100BD0800C2
:0C651400501AA85908ED26FFE40836FADA
:0E6520000886038F828A838BF0EE1273B00D13
:02652E0080D615
:0C653000A85908ED26FAE40836FB08869E
:0D653C00048A828B838CF0E41273B08D8290
:06654900855981D05922A2
:057D48004A616E0B0012
:057D4D004665620B0019
:057D52004DE4720B007E
:057D57004170720B00F9
:057D5C004D61692000EB
:057D61004A756E0B00E5
:057D66004A756C0B00E2
:057D6B004175670B00EB
:057D70005365700B00DB
:057D75004F6B740B00D0
:057D7A004E6F760B00C6
:057D7F0044657A0B00D1
:047D84003F3F3F003E
:037D88002D2D009E
:0A654F00C059858159AA821AEA2476
:08655900F450057582FF804239
:0C656100A859181818B6000AEA907D9797
:06656D0093FBF582803073
:0C657300A859181818740356FB60028029
:01657F001B00
:0C658000A85918181875F064E684ABF0F8
:05658C00BB0002800AC3
:0A659100EA907D9793FBF5828008E5
:08659B00EA907D8B93FAF58272
:0665A300855981D0592248
:0A65A900C059858159C082C083C02B
:0C65B300F0E5812408F581A85908740166
:0E65BF0026FDE40836FE0886078D828E838F47
:0C65CD00F01273C9FA6005EA24F35006CE
:0665D900758200026770EC
:0C65DF00A8590886820886830886F012FE
:0A65EB0073C9FB7005F582026770AA
:0A65F500C005C006C007A85908E55C
:0C65FF00592406F9740226F7E408360956
:0C660B00F70809E6F7E5592406F8868236
:0E6617000886830886F01273C9FDC003C00612
:0E662500C007C0058A8212654FAD821581D074
:0E66330007D006D003C3ED9BE433D007D0069A
:0A664100D005600675820002677044
:0C664B00E5592406F8868208868308863C
:0C665700F01273C9FA7B00E5592404F826
:0E66630074D02AF674073B08F68D828E838F62
:08667100F01273C9FCBC030028
:0C667900500EE5592404F8E624FFF60852
:04668500E634FFF602
:0C668900E5592404F8860508E6C313CD8B
:0C66950013CDC313CD13CDFEE559240432
:0E66A100F8ED26FDEE0836FEC004C005C0066A
:0C66AF007464C0E0E4C0E0E5592404F885
:0B66BB00E5592404F88682088683124B
:0E66C600737FAF82AA8315811581D006D0059F
:0E66D400D004EDC39FFDEE9AFEC004C005C0C9
:0C66E200067490C0E07401C0E0E559248B
:0C66EE0004F8E5592404F886820886832D
:0E66FA0012737FAA82AB8315811581D006D062
:0E67080005D004EA2DFDEB3EFEEC14907DA3BF
:0C67160093FA7B002DFDEB3EFEA8590815
:0E67220086820886830886F01273C9FA7B000F
:0E6730002DF582EB3EF5837407C0E0E4C0E077
:0C673E00127422AA82AB8315811581E53C
:0A674A00592404F8A60208A603E58E
:0C675400592404F8B6000E08B6000AE54F
:09676000592404F87607E408F658
:07676900E5592404F88682C3
:06677000855981D0592279
:0A677600C059858159C082C083C05C
:0C678000F0058105810581A8590874010D
:0E678C0026FDE40836FE0886078D828E838F78
:0E679A00F01273C9FD14FE24F4500690FFFFA8
:0367A8000268750F
:0C67AB00A8590886820886830886F01230
:0767B70073C9FF60028006B8
:0667BE0090FFFF02687568
:0A67C400C006A85908E5592404F99D
:0E67CE00740226F7E4083609F70809E6F7E535
:0C67DC00592404F886820886830886F0A1
:0D67E8001273C9FEC006C007C0068D8212E4
:0E67F500654FAD821581D007D006ED3395E0DB
:0E680300FE7A00C3ED9FEE64808AF063F080A1
:0D68110095F0E433D006600590FFFF80573E
:0C681E00A8590886820886830886F012BC
:0A682A0073C9FA7B001ABAFF011BC4
:026834008E04D0
:0C683600EC24FF5036E5592404F886825B
:0E6842000886830886F01273C9FDC002C003E9
:0E685000C004C0058C8212654FAD821581D048
:0E685E0004D003D002ED3395E0FEED2AFAEEF1
:05686C003BFB1C80C590
:046871008A828B8309
:06687500855981D0592273
:0D687B00AA82AB83ACF0C002C003C00412BF
:0E68880068A5E582D004D003D002601074032E
:0E6896002AFAE43BFB8A828B838CF002692E87
:0168A40022D1
:0E68A500AA82AB83ACF074022AFDE43BFE8CA9
:0E68B300078D828E838FF01273C904F88D82D8
:0A68C1008E838FF01273B0B83C0014
:0E68CB00405D8D828E838FF0E41273B07401F5
:0E68D9002AFDE43BFE8C078D828E838FF01229
:0E68E70073C904F88D828E838FF01273B0B8DF
:0268F5003C0065
:0E68F70040318D828E838FF0E41273B08A825E
:0E6905008B838CF01273C904FD8A828B838C05
:07691300F01273B0BD180083
:0E691A00400E8A828B838CF0E41273B075827B
:0269280001224A
:04692A007582002250
:0A692E00C059E581F5592406F581F2
:0E693800AA82AB83ACF01273C904FD8A828B75
:0C694600838CF01273B0E5592404F8743F
:0C695200022AF6E43B08F608A604E5590A
:0E695E002404F886820886830886F01273C926
:0C696C00FFA8590874012AF6E43B08F665
:0C69780008A604A8590886820886830837
:0E69840086F01273C9FEC002C003C004C00535
:0E699200C0078E8212654FAE821581D005D0EF
:0E69A00004D003D002C3EE9D50618A828B8327
:0C69AE008CF074011273B0A859088682A6
:0C69BA000886830886F01273C904FAA84E
:0C69C600590886820886830886F0EA12D1
:0C69D20073B024F35033A85908868208E3
:0C69DE0086830886F074011273B0E5593E
:0E69EA002404F886820886830886F01273C99A
:0C69F80004FAE5592404F886820886831E
:076A04000886F0EA1273B0EE
:066A0B00855981D05922DB
:0A6A1100C059858159C082C083C0BE
:0C6A1B00F00581A85908740326FDE4086A
:0E6A270036FE08860774012DFAE43EFB8F044C
:0C6A35008A828B838CF0E5592404F8124F
:0C6A410073C9F6E5592404F8E624FC5063
:096A4D0010E5592404F8B60A0012
:086A56005006758201026B5F1E
:0D6A5E008D828E838FF0C002C003C0041231
:0E6A6B0065A9AD82D004D003D002BD07027D24
:016A7900001C
:0E6A7A008A828B838CF01273C9FEBE036DC03E
:0C6A880005A85908740326FFE40836FD39
:0E6A94000886028F828D838AF01273C9FABAC7
:026AA2001900D9
:0E6AA400D00540187B008D047F00EAC39CFAE9
:0E6AB200EB9FFBC3EA9419EB648094805006BE
:066AC000758200026B5F0D
:0C6AC600BD0025A85908868208868308B8
:096AD20086F01273C9FABA020041
:086ADB005006758200026B5F9A
:036AE300BA0300F3
:086AE6005006758202026B5F8D
:066AEE00758201026B5FDE
:0C6AF400BE0A65A85908740326FAE408DD
:0E6B000036FB0886048A828B838CF01273C9E0
:046B0E00FABA1900B6
:0E6B120040187B008D047E00EAC39CFAEB9EC7
:0C6B2000FBC3EA9419EB648094805005DC
:056B2C00758201802EBE
:0C6B3100BD0023A859088682088683084E
:096B3D0086F01273C9FABA0200D5
:076B46005005758201801269
:036B4D00BA030088
:076B50005005758203800867
:056B57007582008003BF
:036B5C007582003F
:066B5F00855981D0592286
:0A6B6500C059858159C082C083C069
:0C6B6F00F0E581240AF581A859087402A1
:0E6B7B0026FDE40836FE0886078D828E838F85
:086B8900F01273C9FDBDC80044
:056B910040030270C08A
:0A6B9600A85908A85908868208864D
:0C6BA000830886F0126776AD82AE83E5B4
:0A6BAC00592405F8A60508A606E521
:0C6BB600592405F8B6FF0A08B6FF067562
:056BC20082010270E5F4
:0C6BC700A85908740226FFE40836FD08F7
:0C6BD30086068F828D838EF0E559240A1F
:0C6BDF00F81273C9F6E559240AF886057F
:0E6BEB007E0074642DFFE43EFAC002C005C0B7
:0E6BF90006C0077413C0E0E4C0E08F828A83F8
:0E6C0700127422AB82AC8315811581D007D0A8
:0C6C150006D005D002E5592404F8A603BF
:0E6C21005307037A0074672DF582E43EF58375
:0E6C2F00C0077407C0E0E4C0E0127422AA821D
:0C6C3D00AB8315811581D0078A06E5594C
:066C4900240AF8B6640005
:056C4F004003026CD2BD
:0C6C5400E5592404F8E675F013A4241898
:0E6C6000F582E435F0F583C006C007741EC04F
:0E6C6E00E0E4C0E01273E5AA82AB8315811545
:0E6C7C0081D007D0068F03E4FCCB25E0CB339C
:0E6C8A00FC8E07E4FDCF25E0CF33CF25E0CF11
:0E6C980033FDEF2BFBED3CFCEA75F006A4FD8E
:0E6CA600AEF0ED2BFBEE3CFC8B828C83A3A3A7
:0D6CB400A3A3A3C0027407C0E0E4C0E01277
:0E6CC10073E5AB82AC8315811581D0028B0682
:036CCF00026D4F04
:0C6CD200E5592404F8E675F013A424181A
:0E6CDE00F582E435F0F583C006C007741EC0D1
:0E6CEC00E0E4C0E01273E5AB82AC83158115C5
:0E6CFA0081D007D0068B028F03E4FCCB25E08F
:0E6D0800CB33FC8E07E4FDCF25E0CF33CF2543
:0E6D1600E0CF33FDEF2BFBED3CFCEA75F00601
:0E6D2400A4FDAEF0ED2BFBEE3CFC74062BF54F
:0E6D320082E43CF583C0027407C0E0E4C0E0D8
:0E6D40001273E5AB82AC8315811581D0028BF6
:016D4E00063E
:0E6D4F008A037C0074162BFBE43CFC8E077D4F
:0E6D5D0000EF2BFBED3CFCC3741F9B74808C7D
:0C6D6B00F063F08095F04038E5592407F3
:0C6D7700F874162AFBEE2BA6E0E5592468
:0D6D830007FB74012BF8760374022BF8E572
:0C6D900059240AF9E7F67C007F408B8252
:0E6D9C008C838FF0126776AB82AC838B028003
:016DAA004F99
:0C6DAB00E5592407F8EE2A24F7FBF686D1
:086DB70004BB1A0476138012DC
:0C6DBF00BC190FBA1C0CE5592404F9E7BC
:066DCB0024F550027612CF
:0C6DD100E5592407FB74012BF8760474CC
:0C6DDD00022BF8E559240AF9E7F67C00C7
:0E6DE9007F408B828C838FF0126776AB82AC7A
:036DF700838B0289
:0C6DFA00A85908740126FBE40836FC08C8
:0E6E060086078B828C838FF01273C9FBE4BB6E
:036E140001010475
:0C6E1700FC6018A85908868208868308D1
:0D6E230086F01273C9FFBF010675820202DE
:026E300070E50B
:0C6E3200EC6018A85908868208868308C6
:0D6E3E0086F01273C9FCBC060675820302C3
:026E4B0070E5F0
:0E6E4D00C0038A047F00EC24CCFBEF34FFFD71
:0C6E5B00E5592405F8E6B5030908E6B582
:066E670005047401800126
:016E6D00E440
:0A6E6E00D00360067582040270E58F
:0C6E7800EC24D0FDEF34FFFEE5592405AA
:0C6E8400F8E6B5050708E6B50602800236
:026E900080067A
:066E92007582050270E5A7
:0C6E9800EC24D1FDEF34FFFEE559240589
:0C6EA400F8E6B5050708E6B50602800216
:026EB00080065A
:066EB2007582060270E586
:0C6EB800EC24D2FDEF34FFFEE559240568
:0C6EC400F8E6B5050708E6B506028002F6
:026ED00080063A
:066ED2007582070270E565
:0C6ED800EC24FDFDEF34FFFEE55924051D
:0C6EE400F8E6B5050708E6B506028002D6
:026EF00080061A
:066EF2007582080270E544
:0C6EF800EC24FEFDEF34FFFEE5592405FC
:0C6F0400F8E6B5050708E6B506028002B5
:026F10008006F9
:066F12007582090270E522
:0C6F1800E5592405F8E6B5040708E6B5C5
:046F240007028002DE
:026F28008006E1
:066F2A0075820A0270E509
:0C6F300074012CFDE43FFEE5592405F837
:0B6F3C00E6B5050708E6B50602800276
:026F47008006C2
:066F490075820B0270E5E9
:0C6F4F00BB0518A8590886820886830834
:0D6F5B0086F01273C9FDBD010675820C029F
:026F680070E5D2
:0C6F6A0074272CFDE43FFEE5592405F8D7
:0B6F7600E6B5050708E6B5060280023C
:026F8100800688
:066F830075820D0270E5AD
:0C6F890074312CFDE43FFEE5592405F8AE
:0B6F9500E6B5050708E6B5060280021D
:026FA000800669
:066FA20075820E0270E58D
:0C6FA80074322CFDE43FFEE5592405F88E
:0B6FB400E6B5050708E6B506028002FE
:026FBF0080064A
:066FC10075820F0270E56D
:0C6FC700743C2CFCE43FFFE5592405F865
:0B6FD300E6B5040708E6B507028002DF
:026FDE0080062B
:066FE0007582100270E54D
:0C6FE600BB0818A859088682088683089A
:0D6FF20086F01273C9FCBC0F0675821102F7
:026FFF0070E53B
:0C700100BB0A18A859088682088683087C
:0D700D0086F01273C9FCBC030675821202E6
:02701A0070E51F
:0C701C00BB0B18A8590886820886830860
:0D70280086F01273C9FCBC010675821302CC
:0270350070E504
:05703700E4BB0C0104A4
:0C703C00FB6018A85908868208868308AB
:0D70480086F01273C9FCBC060675821402A6
:0270550070E5E4
:0C705700EB6018A85908868208868308A0
:0D70630086F01273C9FCBC18067582150278
:0270700070E5C9
:0C707200EB6017A8590886820886830886
:0E707E0086F01273C9FCBC1905758216805984
:0C708C00EB6017A859088682088683086C
:0E70980086F01273C9FCBC1A05758217803F82
:0C70A600EB6017A8590886820886830852
:0E70B20086F01273C9FBBB1F0575821880257E
:0A70C000A85908A85908868208861E
:0E70CA00830886F01265A9AB828B02BA06021B
:0270D800800333
:0370DA00BA0705ED
:0570DD00758201800333
:0370E200758200B4
:0670E500855981D05922FB
:0A70EB00E582FA24E75003027194D5
:0D70F500EA240983C0E0EA241C83C0E022E5
:02710200949067
:0271040034381D
:027106003C400B
:027108004448F9
:02710A004C50E7
:02710C005458D5
:02710E005C60C3
:027110006468B1
:027112006C709F
:0271140074788D
:027116007C807B
:02711800848869
:01711A008CE8
:02711B00717190
:02711D0071718E
:02711F0071718C
:0271210071718A
:02712300717188
:02712500717186
:02712700717184
:02712900717182
:02712B00717180
:02712D0071717E
:02712F0071717C
:0271310071717A
:0171330071EA
:04713400758201223D
:04713800758200223A
:04713C007582002236
:047140007582002232
:04714400758200222E
:04714800758200222A
:04714C007582002226
:047150007582012221
:04715400758201221D
:047158007582012219
:04715C007582012215
:047160007582012211
:04716400758201220D
:047168007582012209
:04716C007582012205
:047170007582002202
:0471740075820122FD
:0471780075820122F9
:04717C0075820022F6
:0471800075820022F2
:0471840075820122ED
:0471880075820122E9
:04718C0075820022E6
:0471900075820022E2
:0471940075820022DE
:0A719800E582FA24E7500302724179
:0D71A200EA240983C0E0EA241C83C0E02237
:0271AF00413D60
:0271B100E1E516
:0271B300E9ED04
:0271B500F1F5F2
:0271B700F9FDE0
:0271B9000105CE
:0271BB00090DBC
:0271BD001115AA
:0271BF00191D98
:0271C100212586
:0271C300292D74
:0271C500313562
:0171C700398E
:0271C8007272E1
:0271CA007171E1
:0271CC007171DF
:0271CE007171DD
:0271D0007171DB
:0271D2007272D7
:0271D4007272D5
:0271D6007272D3
:0271D8007272D1
:0271DA007272CF
:0271DC007272CD
:0271DE007272CB
:0171E000723C
:0471E100907DAF22CC
:0471E500907DB722C0
:0471E900907DCB22A8
:0471ED00907DDF2290
:0471F100907DED227E
:0471F500907E042262
:0471F900907E15224D
:0471FD00907E262238
:04720100907E332226
:04720500907E422213
:04720900907E502201
:04720D00907E6022ED
:04721100907E7722D2
:04721500907E8822BD
:04721900907E9822A9
:04721D00907EA72296
:04722100907EBC227D
:04722500907ECD2268
:04722900907EDD2254
:04722D00907EE62247
:04723100907EF42235
:04723500907F0E2216
:04723900907F2822F8
:04723D00907F3422E8
:04724100907F4122D7
:0A724500C059858159C082C083C082
:0C724F00F0058105810581E55924FBF85C
:0C725B008605088606088607A8590886E4
:0E726700820886830886F01273C9FA8D828E23
:0C727500838FF01273B0E5592404F87404
:0C728100012DF6E43E08F608A607A85907
:0E728D0008740126FAE40836FB0886048A829B
:0C729B008B838CF01273C9FAE5592404AF
:0E72A700F886820886830886F0EA1273B074B7
:0C72B500022DFDE43EFEA85908740226DC
:0E72C100FAE40836FB0886048A828B838CF080
:0E72CF001273C9FA8D828E838FF01273B08510
:0572DD005981D0592287
:0A72E200C059858159C082C083C0E5
:0C72EC00F0058105810581E55924FBF8BF
:0C72F8008605088606088607A859088647
:0E730400820886830886F01273C9FA8D828E85
:0C731200838FF01273B0E5592404F87466
:0C731E00012DF6E43E08F608A607A85969
:0E732A0008740126FAE40836FB0886048A82FD
:0C7338008B838CF01273C9FAE559240411
:0E734400F886820886830886F0EA1273B07419
:0C735200022DFDE43EFEA859087402263E
:0E735E00FAE40836FB0886048A828B838CF0E2
:0E736C001273C9FA8D828E838FF01273B08572
:05737A005981D05922E9
:0C7D8B001F1C1F1E1F1E1F1F1E1F1E1F7F
:0C7D97001F1D1F1E1F1E1F1F1E1F1E1F72
:0C7DA300000302050003050104060204B1
:087DAF004E65756A61687200FF
:0E7DB7004865696C69672D0A447265690A6B3C
:067DC500F66E696765001F
:0E7DCB005765696265722D0A666173742D0A30
:067DD9006E616368740096
:0E7DDF00526F73656E2D0A6D6F6E74616700D2
:0E7DED00466173742D0A6E61636874732D0A0B
:097DFB006469656E737461670030
:0E7E04004173636865722D0A6D697474776F3F
:037E1200636800A2
:0E7E15004772FC6E646F6E2D0A6E6572737498
:037E230061670094
:0D7E26004B6172667265692D0A7461670018
:0E7E33004F737465722D0A736F6E6E74616703
:017E41000040
:0E7E42004F737465722D0A6D6F6E7461670068
:0E7E5000546167206465722D0A417262656993
:027E5E007400AE
:0E7E6000436872697374692D0A48696D6D6517
:097E6E006C2D0A66616872740053
:0E7E77005066696E6773742D0A736F6E6E74B9
:037E850061670032
:0E7E88005066696E6773742D0A6D6F6E7461BB
:027E9600670083
:0E7E980046726F6E2D0A6C656963686E616DCF
:017EA60000DB
:0E7EA7004D617269E42D0A48696D6D656C2DA0
:077EB5000A666168727400A7
:0E7EBC00546167206465722D0A45696E686521
:037ECA00697400D8
:0E7ECD00416C6C65722D0A6865696C696765A9
:027EDB006E0037
:097EDD004E696B6F6C6175730056
:0E7EE6004865696C69672D0A6162656E64000B
:0E7EF400312E20576569682D0A6E616368742F
:0C7F0200732D0A66656965727461670082
:0E7F0E00322E20576569682D0A6E6163687413
:0C7F1C00732D0A66656965727461670068
:0C7F280053696C2D0A7665737465720055
:0D7F3400576F6368656E2D0A656E64650009
:087F41005765726B7461670063
:0A737F00E58124FEF886011886005F
:057389007A10E4FBFC9A
:0E738E00E58225E0F582E58333F583EB33FBE2
:0E739C00EC33FCEB98F5F0EC994006FCABF0FE
:0373AA004382011A
:0373AD00DADF2202
:06004D00E478FFF6D8FD87
:08002B007900E94400601B7A32
:0500330000907F4978F8
:030038000075A0B0
:0A003B0000E493F2A308B8000205E8
:08004500A0D9F4DAF275A0FF66
:0E73B00020F71030F6118883A88220F507F62A
:0573BE00A883758300A7
:0173C30022A7
:0373C400F280F75D
:0273C700F022B2
:080053007800E84400600A791E
:03005B000075A08D
:06005E0000E4F309D8FCE8
:080064007800E84400600C790B
:0B006C0000900000E4F0A3D8FCD9FADB
:03001E0075815990
:0A002100127467E58260030200FE1E
:0E73C90020F71430F6148883A88220F507E61A
:0673D700A883758300226B
:0373DD00E280F754
:0373E000E4932211
:0273E300E022A6
:0E73E500C2D5E58330E70DD2D5E4C39582F51D
:0673F30082E49583F5839E
:0E73F900E58124FEF8E630E70918E4C396F6B5
:04740700E40896F609
:0E740B00860118860012742C30D50BE4C39550
:0874190082F582E49583F583FE
:017421002248
:0A742200E58124FEF88601188600BB
:06742C00E84960367A0118
:0E743200E825E0F8E933400EF9E58298E5839D
:067440009940030A80ECF4
:02744600C3E998
:0574480013F9E813F840
:0E744D00C3E58298F5F0E583994005F5838547
:02745B00F082BD
:09745D00C3E913F9E813F8DAE7BA
:017466002203
:047467007582002208
:00000001FF
